:100000000C94E40B0C940C0C0C940C0C0C940C0C39
:100010000C940C0C0C9462120C940C0C0C940C0CA4
:100020000C940C0C0C940C0C0C940C0C0C940C0CF0
:100030000C940C0C0C940C0C0C940C0C0C940C0CE0
:100040000C9419200C940C0C0C940C0C0C940C0CAF
:100050000C940C0C0C940C0C0C940C0C0C940C0CC0
:100060000C940C0C0C940C0C0C1B651B791B851B45
:10007000891B921B9A1B9E1BA71BB31B091B031BEF
:1000800088228822882250235023B022C522DC22D5
:10009000E922F722122350235023502338235F00F4
:1000A000040305050405061515FFFB0EFC0EFD02F5
:1000B0008B05432006002034012109C32D44E107AC
:1000C00062062212C8245661644264426442644259
:1000D000644264002322CC25744B444C444A46E6D7
:1000E00060E4604695889888CC01C5018D88988821
:1000F000948C9488140024202AA6632BAEE62064F6
:10010000826224C224C8CACCAC2AC224C22462E2BD
:1001100020C62E320800252BD225A4852ECA4A4897
:100120008D94904C989088D8C884A089C8948C8865
:100130008464888C9C888C988C3219555255722313
:10014000002621CE2584A7EE206C666A666A64CEFE
:1001500092D06682624464664264A8646AE880CA97
:1001600082002709C32C46A1421700280F246A43A6
:10017000456285C4FE89C8C488002913246A4341A6
:1001800044646244C9C42E4424568888002A11E875
:10019000E8654344864AE620468A464402002B0E20
:1001A0008C31A42D3657070FC66273052C0BA4A4FF
:1001B000336385C48408002D0865243DE141002E89
:1001C00008632834E140002F0FE6E54B4937426AC7
:1001D00084D4086923043013CA255C87E846486242
:1001E000C83F9A10123908A201310CC6295C67E297
:1001F000C06266FF013215CA255CA7E62044C868C4
:100200006ED91815ABB1B18303033314CA255CA5AD
:10021000E864666E5155E13AA39391A31A00341A2B
:10022000CB255C8BAC95C4D0C490C8CCC88CCCC852
:10023000CCC8C183B0C125003519CA255CE140E2B4
:1002400040626EDD41C881C490E09C91CDC8510DE3
:1002500000361BCA255C87EA4448446E4EA2E4403F
:10026000624862C8D18490C841100D003715CA2574
:100270005CE181DDD8DC18D9DCD8DCD8DC18D914F5
:10028000003817CA255CC5E62062C891C891CDC860
:10029000C490471307312600391CCA255C87E864DF
:1002A00048624862C8E884E24046644E6248446658
:1002B000E4A806003A0A432D3CE140F840003B0E1A
:1002C00084A533637B900989091111003C0E4C71A0
:1002D000A437706E6CA5F0DA61013D0BACF0A4E1BF
:1002E00083E18307033E104C71A421787678A9DC62
:1002F000D8DC9C28003F14C9255CA5E6426822682A
:100300006C6A4C3BF51072420040355326ABCFF47B
:10031000808E8C689264E66264E420C46466C4647F
:1003200066C46466C46466C46466C464844464E485
:10033000A0648684681E842CF260F6200A00411EA8
:10034000CE21748B94B4D070426E646C646C466A37
:1003500068E860E880646C646C627000421FCB25C2
:100360006CE120E6406468626862686266E420E6E8
:1003700040644A62CAD581C5410C004318CD257C32
:10038000A9EC40666A446C6274CF28C44686680E45
:10039000C48A004418CC2574E120E8606488626A4D
:1003A00062CC5F4D0C511C8C1C04014512CA2564A3
:1003B000E103B9ED0E240E24E6B63B3830460DC9F4
:1003C000255CE1B3CD0E9EED1900471DCD257CC9FE
:1003D000EC40666A62CC74D181D0819CDDC4D804C3
:1003E000D5C801D1410400480ECC257461CCCF0E94
:1003F0003E10F3B3014907C3252CE11F4A0FCA255C
:10040000646F7F67647442711053034B1DCB256C7E
:1004100061E886626664CDC49095D5D1C4D0C8CC5D
:1004200008C90CC5D0C4D4004C0CCA255C616EFF51
:10043000BB8303034D25D02594A1EC60EC80E8A09C
:10044000E8A048C24266C26264C26244C44462C454
:10045000931A1B1A1B1A9BA1014E21CD257C81ECFE
:1004600020EA20EA40C862C662C664C464C466C2A8
:1004700066C2E840E840EA20AA004F1ACE2584C9A7
:10048000EC60666A466E625062D0872272235343E4
:10049000076346005016CB256CE120E66062686277
:1004A000CAA38983898398C11D025120CF258CC995
:1004B000EE406A91DCC8A0C8E0C4E0C4E0C4E0C477
:1004C000A08CDCCC14D181D101015215CB256CE17B
:1004D00040E46062CAAB83928389A189299F095352
:1004E0001BCC2574C7EA20466A626A62D2EE20EC11
:1004F00020AED4CC4CE440CA0600540CCC2574E1A8
:1005000083A1C9FDAF005510CC257461CCFFD9C4BF
:10051000D0CC41940D00561ECE217C816E626E625D
:100520008C646A666A66686A666A668A626E62CEA9
:10053000B2251500572ED421A48188C510D1C8102A
:10054000D1C88CCDC88CCD122543234A8626462699
:1005500086264626A6248424C48ACA8ACA8AEAC66B
:100560008600581ACC2574616C62688466C99459F7
:10057000213BAB09A29199A189A9B3015914CC21BE
:100580006C816A62886466A389A989B13ACA7D04CC
:100590005A15CB256CE360E2608E8C6E8E8C1D1933
:1005A000B3B28307015B0C452A43E1C064FF4F0EE1
:1005B000065C11E6E54B41484A489590AA2821552A
:1005C000420A5D0C452A43E16064FF4F0E0C5E1643
:1005D0008A35A449505D4858489488506EC242C23A
:1005E00022C406035F084A6053E18101600A851C4A
:1005F0002F6166464800611249255CA5E68066C603
:10060000E280C6CD41C988006213CA2564616E17B5
:10061000240712437E247120314102631049255C76
:10062000A5E662C6D91A9B899B12006411CA25648B
:100630006F27141307457E34712042316513492515
:100640005C87E662C6E6E0C1D8CCC44148090066D2
:100650000FC7254487A46468E4E064683F01671914
:10066000CA25638562E24062C6C847130722147335
:1006700013421307312600680EC9255C616C1714FC
:100680000735FECD00690BC3252CE140E6E00301F0
:100690006A0D442A3B63AB89FD170713006B14C92D
:1006A000255C616C2727134B6CDC4C8CAC1899983B
:1006B000196C07C3252CE11F6D1C4F2594618284A2
:1006C000E2E08086C466A866A866A866A866A866F2
:1006D000A86648006E0C49255C6182E2A0C6BF197D
:1006E0006F144A256487E820444862C8A309219111
:1006F00083201A007015CA25636182E44062486253
:10070000C8470715132473DB017111CA256385627D
:10071000E2A0C88F260E4428E676720C4625446176
:10072000E2A06466DF00731249255CA5E42062C67E
:10073000CEAACEE680A60400740EA7254C2968C96F
:10074000C1C9D01ED510750C49255C61C6BF39A83A
:10075000A01876164B215C616A6266646646D1C455
:10076000D0C4948458BB2100772051218C616885C6
:10077000108DC848C91209911911893516134226DE
:100780004535553464443300781449255C6166620C
:10079000446462A66AAAA866628DCD007919CB214D
:1007A0005B616A6266646689D0C4D0C454591DDD39
:1007B000E0BAC129007A0D482554E181D4D05E1DEC
:1007C0001C087B1367EA5269A464684732345244B8
:1007D00053433B2A1A7C07A1EE3AE1037D1267EAF4
:1007E0005261886A68AFC66416ED09CD10007E0DAF
:1007F0006B205D454AE2404286040000005F000530
:100800000506060506073234FFF323F724FA066FC0
:100810000D5620060000C1272D098D21D328F8018F
:10082000082E098751C127F8C0022F2AD129BB2AD7
:100830002B18C14A8C6065AB602546B0122358D98D
:100840002A588911ACC40856B60A565A052B31826B
:1008500095AD82013049D92843EE519AA320249DB9
:10086000A91CE628063AC6918C61286318CB10C6ED
:1008700032C2B18C702C231CCB08C772BF65846355
:1008800019E158863096218C6508431DE2480631EF
:10089000D0410E7398C94808524E5310003118CFFA
:1008A00058412E3A0E5214B2880F4CA1110B49CC6C
:1008B00081CEFFFF1F322FD928432E5AD893A2335F
:1008C000956A200619473A84A18E70A8439EC543B5
:1008D0001E11812898BC742E79A987BCE421108947
:1008E0001FF8031A333DD82843AE59D683223391DB
:1008F0006A1C0611073AC4910C71A4239EE0110FE3
:10090000972C86292E794B6B22228F7848431ED153
:1009100051AE7404041DE238C7A8C86422F4ACE5E3
:1009200000343DDA18416E4BA0F2568ED51A66841B
:100930008319E158863896210E658C231DE34806FD
:100940003990510E6494E318E6CC18E728063AC8AB
:10095000810E62A4837CE01F08DE31CF470035346E
:10096000D828416EA8467DE388E71BC739C25228C4
:10097000528D6A240511073AC4918E60A8239E8B7C
:100980008E72D2118E7404E41CA31A549190B39801
:100990000300364BD928432E529AA3202419AA20AB
:1009A000E520C839C6810E71C89334E4418E73883E
:1009B000A51CA1214770C625168208C520214147E4
:1009C00040941110F5A68E7028431CCA10083A04F2
:1009D000828E8198A34C663A51729A8200372FD842
:1009E00028412EF807A87882473C20020F88C003D0
:1009F00022F080A88740E42110810744E001510FD4
:100A000081C84320F21088BCE4210C00384CD9285E
:100A100043AE611684A652916A242511C841C4913F
:100A20000E71A4431CE910473AC4918E719C832037
:100A3000E5385172DAB2202419A4200339C738D21C
:100A4000118E65846319E158AEF524281D0239889A
:100A5000B84645A813A9C6003947D92843EE599886
:100A6000A3A233158A200619073A86919070A8230D
:100A70001CEA08877A979270A0242065119778C2A3
:100A8000319C7010461CC7288734E49938D0310E49
:100A9000748CE320E42888998C8420E534050100D7
:100AA0000000000000000000000000000000000046
:100AB0000000000000000000000000000000000036
:100AC0000000000000000000000000000000000026
:100AD000000000000000000000005F0004040505A5
:100AE000040506171900FA11FB11FD02ED05FE20A1
:100AF0000600203C012109232E4CE1036309220A50
:100B0000E8A86661887D320023282E26844D8CB0AB
:100B100031C2C40C132388092331E2C4081B234CBF
:100B2000CC98168C860C13234E8CB031C2C48C0228
:100B30002428AC66732D6429342A88849826C4340A
:100B4000A14A043387EC9CB110678298097224048F
:100B50000935C888860D0500253D3526BCA59CB005
:100B600053C3C48812264ACC305162C48912225021
:100B70009488916284080A756284A122D2881C211B
:100B80004AA01051E2868812274694304163468D70
:100B90003A26AE08002627302694C7243A22C406F7
:100BA0000D1B436EC8C0A345CD1019416408154301
:100BB000061D196564182142651C1D212709E3AC37
:100BC0004EE1C108012812856A4B658A21539018AD
:100BD000323F21321B31032913856A4B618C9821E6
:100BE000D30C997F3164122143002A1A292D7E45A6
:100BF000842011824408093264C99020220489109B
:100C0000244208002B0ECE35C42D74BC7BD02C742E
:100C1000BC032C0DC5643B65C4902162840C012D7E
:100C200008662445E1C1002E0763283C21012F19E5
:100C300048E6536B943051A38449354A98A851C271
:100C4000A41A254CD4280030172B266CA7D4994918
:100C5000068918657F3562909031634E9501310D9C
:100C6000272A6C69C8032383E6FF0032192C266CFF
:100C7000A954123243468D9C901CB962959123561B
:100C8000EEC1030333182B266CA7500A32A7064E79
:100C900037AA58C9094D9D7182AA0C00341B2C2615
:100CA0006C8D5C65A6468C1A3168C898391934E495
:100CB000C103732367020035182B266C4185160388
:100CC00067514405995303079A32E4049119003699
:100CD0001E2B266C89149A2124068D103845111577
:100CE000644ED96A84A81163C69C2A030037172B67
:100CF000266CE18381E3C88D23378EBA71E4C691F7
:100D00001B471500381A2B266CA7500A32A7AC1ABD
:100D10003166CCA133538CB2D5191289CA00391D62
:100D20002B266CA7D4992946891865D519124A4AE9
:100D30000C1C68CAD09031435011023A09832D3CF3
:100D4000213D98043B10C5A54365F680878C183279
:100D500044C810003C128E75C45928398203098E8C
:100D60001D4D7A34C5023D0BCE34C5E1417BD00F19
:100D70001A3E148E75C4413069D2A3498F1D487044
:100D80002039A282013F192A2664A5108A31234402
:100D90008D9B6C18A961E3044A0F5AA02800403EBD
:100DA000D6E6C2F1F4CA67E50A952443C508224491
:100DB000924C338408924163CC0C1A6366D018338A
:100DC00083C6981934C60C112223C8381963C20C83
:100DD000A131A4C8032A0F86ED726400412130229C
:100DE000848D30E1A2460F92183864E01062648668
:100DF0000D1A368810374EC80D1988720042182C0B
:100E00002A7C41C98A57C7AC1AA144C9A811C36C2E
:100E1000F580451A00431A2E2684C95CA2258488D1
:100E20000C4376761E0F23318CC82042C90C014436
:100E30001A2E2A8C01D91A26A34A8C1B31EEA0BD8A
:100E40003B37625409266B520145102B2A7CE10383
:100E500083337CA0700E1F3C1846102B2A74E103CC
:100E6000833354A1C5C0F91000471C2F2694CB9C96
:100E70002226A5480C3C68782AAD168E1838A2D8D0
:100E80009036CC8E00480E2D2A8C619C7DF7E03B7D
:100E9000FB6E004908232A3CE107064A102B267402
:100EA00071FE4353A60E35496306004B2A2D2A8452
:100EB0006114895143061119436608A111A4469093
:100EC0003A766C04A9218486101A43661091412554
:100ED00046911846004C0D2B2A7461E0FC3F7CF0D3
:100EE00060004D27322AB4C1DC32CE520C52316838
:100EF000848941238C0C216164122393182131C40D
:100F00008C7D54C610214384064E232E2A94A118AA
:100F1000B254A94C0C3231C8C81823638C10313339
:100F2000C40C0943230C8D309519B2024F1C2F2697
:100F30008CAB60AA35A4888C1B41EEA45D1E1C31CD
:100F40006E082932AB121A0250142C2A7C218D9281
:100F500015A38ED9EA85124423E7250051243126B2
:100F60009CAB68BA55148D1B438EC8C82123878C4F
:100F70001C3272C8C82104C78C1B448AD41B570C6E
:100F8000521A2D2A84410D8B07C1CE593662891A17
:100F900016A3480C1B31EC9CED06531C2D267CC976
:100FA00054A23144460D194AD220B27446CF993B1F
:100FB00045624DB24200540D2D267CE1835443E737
:100FC000FF150055122E2A9461A0FD0F8F91204429
:100FD000848D324300562631228C8124899143C866
:100FE00011213768182152A42623438C0CB93103F0
:100FF0004910243174C4D0A3862B0357453722BC33
:1010000081D83012A34A0D19556A08A142440889B3
:101010001044668A3183C68C183368CC8831838843
:101020008811426AC49811C3468C19316CC4981156
:10103000C346881231AE54C152054B1524470800EF
:1010400058232E26848118095243089121336AC8F7
:10105000307426899234776E04A931148D19458233
:10106000D83902591B2D267C61DC2912A3869021D8
:101070003311095223869D2B5872E87C05005A13C0
:101080002C2674E10373E568488E86E4287CF0C062
:10109000005B0BC5EA4AA1C9FCFF13055C1347E6D8
:1010A0005341D428A94649354A56A3A41A25035DBD
:1010B0000BC5EA4A41C9FCFF93065E21CB39BC2B24
:1010C000E4C010E144080B132C4C28318242050A7D
:1010D000154694907021C48D1419005F084C60630C
:1010E000E14102600A84A037618818210261158AF3
:1010F000256CA70C9231E3C69C6863C8D0111249D5
:10110000880862182C267461E4BC28A3840C094268
:10111000C76C7628CD082543C80063148A2564A7C8
:101120000C922187CCCDC8D08821241015016417DA
:101130002C267473DE9418A2820CA263363B4462A0
:101140004C1135440665148B256CA7D49929063DAE
:101150007038D1903143129501661128264CA7882A
:101160009151D33C08326AFE0D00671F2CE672A72E
:10117000C4101564101DB3D921128348AC213272FA
:10118000C4A81164C62432030068112B266C61E0E8
:10119000BC28A2820C2253F6AB01690A23262C211B
:1011A000D98307066A0DC4EA3A639623E6FFC205AF
:1011B000006B1F2B266461E0BC213166C83423C854
:1011C0001C3A3462D0083243880C213286C4200293
:1011D0006C08232634E107066D239325AC6108993A
:1011E00022234C9C285206D12853A34C8D3235CA59
:1011F000D42853A34C8D3235CAD4046E0E8B256C83
:1012000061441115644ED95F0D6F178C2574C71496
:101210009A4123088D1866B34324068D4165060064
:1012200070192CE672610819256546103A66B343B9
:10123000684828195166E45C0271172CE67287C869
:10124000101563121DB3D921126488A82931721EAA
:10125000720E87254C618409376406CD47007314EC
:101260008A2564C50C0A3286909D3277C80C0934F1
:1012700046007410E8255447D4340F828C9AAF0886
:101280001922750E8B256C6194FDD519124A4A0CF2
:1012900076198C216C81D4884124060D213327A333
:1012A000468C1A31CA5C758400772A9321A4811078
:1012B000A11183088D185368C41823638618193345
:1012C00062923123869C3962AA8CA942A50A912395
:1012D000440600781B8B256C810C893143480C3AFD
:1012E000558C5CA93324C60C214166C42002791FA9
:1012F0002CE26281D4884124C8CC091912A3468CFF
:101300001A31CA5C852307121C399014007A108A9E
:1013100025642145326293912236BB07057B14E98F
:10132000AA628B509961F3159942C38A119BDF958C
:10133000227C0822AF42E107057D17E8AA6261140A
:10134000B151F3D9A85263CA0C1A35DF94190500BC
:101350007E0B6C6065859008374400000012000524
:10136000050506050607272A00FA23F724FA0000D8
:10137000000020060080E0132A3254B231B80C6419
:101380004005298C218C53882211825888098C6150
:101390009040840F54C210C5311AB20841A44214BF
:1013A000C71885294881063214002B14BDD360BCB0
:1013B0000D7AFC5FFBC007B236E8F17F0D002C18F8
:1013C0008B91DA931CC42007318A418C6294A21855
:1013D000A53045290C002D09CD906914FC00042E80
:1013E00009C7A8E0137C60012F2AF1945D95158C44
:1013F000602546B0B255B01223588911AC6C15ACBB
:10140000C4085662042B5B052BAD829518C1CA56E1
:10141000C1003049799421F728CD511092CE540E55
:101420007314031DE348C63094318C65086319E1D9
:1014300058463896118E658463B9DF32C2B18C701C
:101440002C4318CB10C63284A10E71248318E820D7
:101450008739CC64240429A729080031186FAC20EF
:10146000171D07290A59C407A6D0888524E640E736
:10147000FFFF0F322F799421172DEC49D1994A356E
:1014800010838C231DC2504738D421CFE2218F888E
:1014900040144C5E3A97BCD4435EF21088C40FFCF3
:1014A000010D333D789421D72CEB41919948350EAD
:1014B0008388031DE2488638D2114FF088874B1687
:1014C000C31497BCA5351191473CA4218FE8285738
:1014D0003A02820E719C63546432117AD6720034DF
:1014E0003D7A8C20B72550792BC76A0D33C2C18C49
:1014F000702C431CCB108732C6918E7124831CC87C
:10150000280732CA710C73668C7314031DE44007FC
:1015100031D2413EF00F04EF98E723003534789440
:10152000203754A3BE71C4F38DE31C612914A9466E
:1015300035928288031DE2484730D411CF454739A0
:10154000E908473A02728E510DAA48C859CC0100E9
:10155000364B7994211729CD5110920C5590721069
:10156000E41CE3408738E4491AF220C739C4528E9C
:10157000D0902338E3120B4184629090A02320CABC
:1015800008887A53473894210E6508041D0241C724
:1015900040CC5126339D28394D4100372F78942077
:1015A00017FC03543CC1231E10810744E00111784D
:1015B00040D44320F21088C00322F080A88740E482
:1015C00021107908445EF2100600384C799421D736
:1015D000300B4253A94835929208E420E2488738FC
:1015E000D2218E7488231DE248C738CE4190729C68
:1015F00028396D5910920C5290819C631CE908C7E0
:1016000032C2B18C702CD77A12940E811C445CA328
:1016100022D4895463003947799421F72CCC51D1D5
:10162000990A4510838C031DC3484838D4110E75A0
:101630008443BD4B4938501290B2884B3CE1184E60
:101640003808238E6394431AF24C1CE818073AC6F4
:1016500071107214C44C464290729A82003A0D077F
:10166000BB20147C60F920FB81050000FDF1F580B2
:1016700005F08005F18032F41011800A101310205B
:10168000113A6614B60AA2270011C02111C1021135
:10169000C7C012C5313C15CB392C00340213CF0022
:1016A000813013E884117A12EA6600102911360895
:1016B000142A000000EF142B0000013F102CF5004D
:1016C00000000000240027002A0000000000250080
:1016D00028002B000000000023002600290004043D
:1016E00004040404040402020202020203030303CA
:1016F00003030102040810204080010204081020A6
:10170000010204081020000000080002010000038C
:1017100004070000000000000000F4113608102A41
:10172000A00000A0FF006200EF102BB80100B0FF86
:101730000062013F102C7000F410101028F500F426
:10174000113688113688102AA00000A0FF00A000E2
:1017500000A0FF00102BB80100B0FF0062013F1095
:101760002C7000F4113648113648102AA00000A051
:10177000FF006200EF102BB80100B0FF0062013FD4
:10178000102C7000F4113608102AA00000A0FF00F1
:10179000A00000A0FF00102BB80100B0FF00620104
:1017A0003F102C7000F4113608102AA00000A0FF92
:1017B000006200EF102BB80100B0FF0062013F1083
:1017C0002C700000062F022F11241FBECFEFD8E08F
:1017D000DEBFCDBF12E0A0E0B1E0EEE9F8E602C066
:1017E00005900D92A034B107D9F723E0A0E4B2E050
:1017F00001C01D92AC35B207E1F71BE0C3EEDBE0A0
:1018000004C02197FE010E94E72FC23ED107C9F70D
:101810000E94F0250C9442340C9400000C94F53393
:101820008AED9AE00E94681685E090E09093490363
:10183000809348038CE890E090934B0380934A0395
:101840008091070190910801019719F487EF91E0C9
:1018500002C086E092E00C9466160F931F9380916D
:101860004C0290914D02892B21F540910901509134
:101870000A0160910B0170910C01809144029091DA
:101880004502A0914602B09147028A019B01080FD0
:10189000191F2A1F3B1FC901B80100934002109372
:1018A000410220934202309343020E94FC320E9484
:1018B000861380914C0290914D02019791F54091D1
:1018C000090150910A0160910B0170910C01809106
:1018D000440290914502A0914602B0914702480F00
:1018E000591F6A1F7B1F8091480290914902A09165
:1018F0004A02B0914B028A019B01080F191F2A1F4F
:101900003B1FC901B801009340021093410220938C
:101910004202309343020E94FC321F910F910C94BB
:1019200086131F910F910895FF920F931F93CF93EA
:10193000DF938DE593E10E946816C0917202D09109
:101940007302F09069028E0108501109C8010E94CB
:101950007B18F81671F18FEF8093A1028AEA8093C9
:10196000A2021092A30224E230E04CE150E067E2D0
:1019700070E083E190E00E943C1783E190E0909357
:101980004903809348038BE490E090934B0380934A
:101990004A031092A1021092A2021092A302C8015F
:1019A0000E947B180E94DB17C8010E947B1880935D
:1019B00069028091090190910A01A0910B01B091F7
:1019C0000C0180389649A849B10594F48FEF8093B3
:1019D000A1028AEA8093A2021092A30224E230E0DC
:1019E0004CE150E067E270E083E190E00E943C1738
:1019F000F09068028E0107501109C8010E947B18FF
:101A0000F81671F18FEF8093A1028AEA8093A20207
:101A10001092A30224E230E04CE150E067E270E073
:101A20008FE290E00E943C178FE290E09093490390
:101A3000809348038BE490E090934B0380934A0398
:101A40001092A1021092A2021092A302C8010E9459
:101A50007B180E94DB17C8010E947B1880936802E4
:101A60008091090190910A01A0910B01B0910C01A4
:101A700080349244AF40B105A4F08BE490E09093A1
:101A800049038093480390934B0380934A03109239
:101A9000A1021092A2021092A30285E192E00E949C
:101AA00066168091090190910A01A0910B01B091F5
:101AB0000C0180349244AF40B10594F48FEF8093D1
:101AC000A1028AEA8093A2021092A30224E230E0EB
:101AD0004FE050E067E270E08BE490E00E943C173A
:101AE000F09067028E0106501109C8010E947B1810
:101AF000F81671F18FEF8093A1028AEA8093A20217
:101B00001092A30224E230E04CE150E067E270E082
:101B10008AE590E00E943C178AE590E090934903A3
:101B2000809348038BE490E090934B0380934A03A7
:101B30001092A1021092A2021092A302C8010E9468
:101B40007B180E94DB17C8010E947B1880936702F4
:101B50008091090190910A01A0910B01B0910C01B3
:101B6000803A9648A140B10594F48FEF8093A1028A
:101B70008AEA8093A2021092A30224E230E04CE1B0
:101B800050E067E270E08AE590E00E943C17F09038
:101B900066028E0105501109C8010E947B18F816D3
:101BA00071F18FEF8093A1028AEA8093A2021092D2
:101BB000A30224E230E04CE150E067E270E086E707
:101BC00090E00E943C1786E790E090934903809351
:101BD00048038BE490E090934B0380934A03109268
:101BE000A1021092A2021092A302C8010E947B18C7
:101BF0000E94DB17C8010E947B18809366028091C7
:101C0000090190910A01A0910B01B0910C01803162
:101C10009742A105B10594F48FEF8093A1028AEA5F
:101C20008093A2021092A30224E230E04CE150E043
:101C300067E270E086E790E00E943C17F090650252
:101C40008E0104501109C8010E947B18F81671F129
:101C50008FEF8093A1028AEA8093A2021092A302DE
:101C600024E230E04CE150E067E270E082E990E08D
:101C70000E943C1782E990E09093490380934803C7
:101C80008BE490E090934B0380934A031092A1025F
:101C90001092A2021092A302C8010E947B180E9417
:101CA000DB17C8010E947B188093650280910901AF
:101CB00090910A01A0910B01B0910C01883E9340D4
:101CC000A105B105B4F08EEA90E0909349038093AA
:101CD00048038BE490E090934B0380934A03109267
:101CE000A1021092A2021092A30285E192E00E944A
:101CF00066168091090190910A01A0910B01B091A3
:101D00000C01883E9340A105B10594F48FEF8093B8
:101D1000A1028AEA8093A2021092A30224E230E098
:101D20004FE050E067E270E08EEA90E00E943C17DE
:101D3000F09064028E0103501109C8010E947B18C3
:101D4000F81671F18FEF8093A1028AEA8093A202C4
:101D50001092A30224E230E04CE150E067E270E030
:101D60008DEB90E00E943C178DEB90E0909349033F
:101D7000809348038BE490E090934B0380934A0355
:101D80001092A1021092A2021092A302C8010E9416
:101D90007B180E94DB17C8010E947B1880936402A5
:101DA0008091090190910A01A0910B01B0910C0161
:101DB00084369105A105B10594F48FEF8093A102BB
:101DC0008AEA8093A2021092A30224E230E04CE15E
:101DD00050E067E270E08DEB90E00E943C171091BC
:101DE00063022297CE010E947B18181771F18FEFC2
:101DF0008093A1028AEA8093A2021092A30224E2B5
:101E000030E04CE150E067E270E089ED90E00E9444
:101E10003C1789ED90E090934903809348038BE44D
:101E200090E090934B0380934A031092A10210928A
:101E3000A2021092A302CE010E947B180E94DB171F
:101E4000CE010E947B1880936302DF91CF911F9196
:101E50000F91FF9008958FEF8093A1028AEA8093FB
:101E6000A20286E98093A30227E130E04CE350E030
:101E700064E270E08BEF90E00E9410188EE990E031
:101E80000E94681686EE8093A1021092A20288EC4E
:101E90008093A30281EF90E09093490380934803DD
:101EA00087E390E090934B0380934A038091110164
:101EB00090911201A0911301B09114010197A10515
:101EC000B10581F48AE090E0A0E0B0E080930D01DC
:101ED00090930E01A0930F01B093100187E192E05F
:101EE0000E9466168091110190911201A091130138
:101EF000B09114010297A105B10581F484E690E048
:101F0000A0E0B0E080930D0190930E01A0930F012B
:101F1000B09310018FE192E00E946616809111014A
:101F200090911201A0911301B09114010397A105A2
:101F3000B10581F484EF91E0A0E0B0E080930D0161
:101F400090930E01A0930F01B093100187E292E0ED
:101F50000E9466168091110190911201A0911301C7
:101F6000B09114010497A105B10581F488EE93E0C6
:101F7000A0E0B0E080930D0190930E01A0930F01BB
:101F8000B09310018FE292E00E94661680911101D9
:101F900090911201A0911301B09114010597A10530
:101FA000B10581F480E197E2A0E0B0E080930D01FB
:101FB00090930E01A0930F01B093100186E392E07D
:101FC0000C9466160895F894809111019091120175
:101FD000A0911301B091140185309105A105B105BF
:101FE00029F481E090E0A0E0B0E003C00196A11DDB
:101FF000B11D8093110190931201A0931301B0932E
:1020000014010E942B0F84E00E942D1F892BD9F30D
:10201000789408958F929F92AF92BF92CF92DF9261
:10202000EF92FF920F931F93CF93F8948AED9AE06B
:102030000E946816CFEFC093A102C093A202C09382
:10204000A30246EEE42EF12CF0924903E0924803FD
:102050000EE610E010934B0300934A038091480270
:1020600090914902A0914A02B0914B02B7FD79C00C
:10207000883E9340A105B105CCF41092A2021092C3
:10208000A30225E130E04CE350E06CE570E08EED1A
:1020900090E00E943C17C093A102C093A202C0939B
:1020A000A302F0924903E09248037AC08FE091E0E6
:1020B00090934903809348038EE392E00E94661652
:1020C000C093A1021092A2021092A30225E130E077
:1020D0004EE250E06CE570E08EED90E00E943C171F
:1020E000C093A102C093A202C093A30260914802D0
:1020F0007091490280914A0290914B0238EE832EF2
:1021000033E0932EA12CB12CA50194010E94C82F7D
:10211000F0924903E092480310934B0300934A0363
:10212000CA01B9010E94E61784EF90E09093490339
:102130008093480310934B0300934A0385E192E098
:102140000E946616609148027091490280914A028D
:1021500090914B02A50194010E94C82F2DEF30E011
:102160008FC089319C4FAF4FBF4F3CF11092A202FC
:102170001092A30225E130E04CE350E06CE570E002
:102180008EED90E00E943C17C093A102C093A20282
:10219000C093A30281EE90E090934903809348039B
:1021A00010934B0300934A036091480270914902D7
:1021B00080914A0290914B0273C08FE091E090931E
:1021C0004903809348038EE392E00E946616C09311
:1021D000A1021092A2021092A30225E130E041E395
:1021E00050E06CE570E08EED90E00E943C1760914D
:1021F00048027091490280914A0290914B0228EE68
:10220000C22E23E0D22EE12CF12CA70196010E94D0
:10221000C82FC093A102C093A202C093A30281EE73
:1022200090E0909349038093480310934B030093ED
:102230004A03CA01B9010E94E61788EF90E0909323
:1022400049038093480310934B0300934A0385E1AD
:1022500092E00E9466166091480270914902809156
:102260004A0290914B02A70196010E94C82F9095B7
:102270008095709561957F4F8F4F9F4F20E031E0A3
:10228000309349032093480310934B0300934A0370
:1022900024E630E040E050E00E94C82FCA01B901B6
:1022A0000E94E6177894CF911F910F91FF90EF90C5
:1022B000DF90CF90BF90AF909F908F900895CF9375
:1022C000DF938AED9AE00E94681680916C029091EB
:1022D0006D02019799F58FEF8093A1028093A2027E
:1022E0001092A30287E090E0909349038093480303
:1022F000C5E1D0E0D0934B03C0934A038FE491E053
:102300000E94661688E490E0909349038093480306
:10231000D0934B03C0934A031092A1021092A202E1
:102320001092A30283E591E00E94661661E087E0C7
:102330000E94561F60E086E00E94561F80916C024A
:1023400090916D02029791F587E090E09093490398
:1023500080934803C5E1D0E0D0934B03C0934A0378
:102360001092A1021092A2021092A3028FE491E0B7
:102370000E94661688E490E0909349038093480396
:10238000D0934B03C0934A031092A1021092A20271
:102390001092A30283E591E00E94661660E087E058
:1023A0000E94561F60E086E00E94561F80916C02DA
:1023B00090916D02039799F587E090E0909349031F
:1023C00080934803C5E1D0E0D0934B03C0934A0308
:1023D0001092A1021092A2021092A3028FE491E047
:1023E0000E9466168FEF8093A1028093A202109242
:1023F000A30288E490E09093490380934803D0932C
:102400004B03C0934A0383E591E00E94661660E0A7
:1024100087E00E94561F61E086E00E94561F80916F
:102420006C0290916D02892B91F587E090E090937A
:10243000490380934803C5E1D0E0D0934B03C09398
:102440004A031092A1021092A2021092A3028FE4FA
:1024500091E00E94661688E490E09093490380938F
:102460004803D0934B03C0934A031092A1021092E9
:10247000A2021092A30283E591E00E94661660E03A
:1024800087E00E94561F60E086E00E94561F809100
:102490006C0290916D0201968430910529F0909321
:1024A0006D0280936C0204C010926D0210926C0257
:1024B0000E942D0C80E00E942D1F892BD9F3DF9103
:1024C000CF9108951F920F920FB60F9211242F9360
:1024D0003F934F935F936F937F938F939F93AF93AC
:1024E000BF93EF93FF9380914C0290914D0201971F
:1024F000B9F50E947817282F882309F470C08091BD
:10250000480290914902A0914A02B0914B022031B9
:1025100079F48C599F4FAF4FBF4F8C3A26E2920708
:10252000A105B105A4F08CEA96E2A0E0B0E00FC0EE
:1025300084569109A109B109853529ED92072FEF3C
:10254000A207B20724F484E599EDAFEFBFEF8093C3
:10255000480290934902A0934A02B0934B023FC0B5
:102560000E947817282F8823D1F18091090190913A
:102570000A01A0910B01B0910C0140910D01509105
:102580000E0160910F0170911001203189F4840FC8
:10259000951FA61FB71F803823EC920729ECA207CE
:1025A00021E0B207A4F080E893ECA9ECB1E00FC001
:1025B000841B950BA60BB70B813A26E8920721E006
:1025C000A207B10524F480EA96E8A1E0B0E0809388
:1025D000090190930A01A0930B01B0930C01FF91A4
:1025E000EF91BF91AF919F918F917F916F915F918B
:1025F0004F913F912F910F900FBE0F901F90189504
:10260000EF92FF920F931F93CF93DF9383E10E948A
:10261000C21F8855924097FD05C090936B0280932E
:102620006A0204C010926B0210926A0280916A02E0
:1026300090916B026CE170E00E94922F6031710505
:102640002CF470936B0260936A0206C08FE090E0F6
:1026500090936B0280936A02E0906A02F0906B02A2
:10266000C1E1CE9D8001CF9D100D11248DEF97E02B
:102670000E9468161092A1021092A2021092A30268
:102680002FE030E02E193F09C29FA001C39F500DDB
:102690001124485D5F4F20E130E064EB70E0C80139
:1026A00089960E943C1788E290E0909349038093BA
:1026B000480388EC90E090934B0380934A03C1E079
:1026C000D0E01FEF80916A0290916B028C179D07FA
:1026D000B4F0CA30D1053CF41092A1021093A202CA
:1026E0001093A30206C01093A1021092A2021092AE
:1026F000A30285EF91E00E9466162196E3CFDF9159
:10270000CF911F910F91FF90EF900895CF92DF929C
:10271000EF92FF92CF93DF9300D0CDB7DEB720E0EA
:1027200030E040E85FE40E9437336B017C01609148
:1027300001017091020180910301909104010E94B6
:10274000FA329B01AC01C701B6010E9401300E9420
:102750007330F62EE82E60E08FE079839A830E9432
:10276000561F8F2D0E9417177981872F0E941717E8
:102770008E2D0E9417179A81892F0E94171780E0CB
:102780000E94171761E08FE00F900F90DF91CF91BB
:10279000FF90EF90DF90CF900C94561FCF92DF9276
:1027A000EF92FF920F931F93CF93DF938C01C0E0C2
:1027B000D0E0C12CD12C7601C8010E940E0CC82A91
:1027C000C330D10531F0FE2CED2CDC2CCC240F5F76
:1027D0001F4F2196C430D10579F7C701B601DF91AB
:1027E000CF911F910F91FF90EF90DF90CF900895C0
:1027F0008F929F92AF92BF92CF92DF92EF92FF9211
:102800001F93CF93DF936B017C015A01C3E0D0E0AB
:102810004E018A0C9B1CC4010E940E0C8C1521F0E9
:102820006C2DC4010E94901DCD2CDE2CEF2CFF24BA
:10283000E7FCFA94219760F7DF91CF911F91FF9009
:10284000EF90DF90CF90BF90AF909F908F900895C2
:10285000CF93DF938330E0F494E0899FE00111246B
:102860006091090170910A0180910B0190910C0116
:10287000AE010E94F813AE01405F5F4F60911101FD
:102880007091120180911301909114010E94F8132C
:1028900060914E0280E290E00E94901D60910501DF
:1028A00082E290E0DF91CF910C94901D80914E02D6
:1028B000833078F424E0829FC00111240E94CE135B
:1028C0006093090170930A0180930B0190930C01AE
:1028D0000EC080E090E00E94CE13609309017093D7
:1028E0000A0180930B0190930C0110924E0280918B
:1028F0004E02833038F490E00496880F991F880FB9
:10290000991F02C080E190E00E94CE1360931101F4
:1029100070931201809313019093140182E290E06E
:102920000E940E0C90E0909306018093050108959B
:10293000E7E7F2E022A5238F23A5248F24A5258F86
:10294000908F878B728F618F0184F285E02D40E03C
:1029500050E064E170E08BE792E00994AF92BF929F
:10296000CF92DF92EF92FF920F93CF93DF93EC0120
:102970007B016A01590100FF10C0B9016E197F097E
:10298000CA018C0F9D1F0E949814B5016C1B7D0B12
:10299000C6018E0D9F1D0E94981401FF10C0B50145
:1029A0006E197F09C6018C1B9D0B0E949814B501FE
:1029B0006C1B7D0BC6018E199F090E94981403FFA2
:1029C00010C0B5016E0D7F1DC6018C0F9D1F0E94AA
:1029D0009814B5016C0F7D1FC6018E0D9F1D0E94BE
:1029E000981402FF19C0B5016E0D7F1DC6018C1B26
:1029F0009D0B0E949814B5016C0F7D1FC6018E19A6
:102A00009F09DF91CF910F91FF90EF90DF90CF90D2
:102A1000BF90AF900C949814DF91CF910F91FF90DD
:102A2000EF90DF90CF90BF90AF9008954F925F925C
:102A30006F927F928F929F92AF92BF92CF92DF92CE
:102A4000EF92FF920F931F93CF93DF932C014B01D3
:102A5000EA01122F81E090E07C01E41AF50ACC240F
:102A6000DD24C41AD50ACC0CDD1C022F9B01A20167
:102A7000BE0180E090E00E94AE14A12CB12C66242F
:102A80006394712CAC16BD06C4F4F7FC06C0219704
:102A900082E0C80ED11CEC0CFD1C8FEFA81AB80AFE
:102AA00082E0680E711CE60CF71C012F9401A20154
:102AB000BE01C5010E94AE14E5CFDF91CF911F91F9
:102AC0000F91FF90EF90DF90CF90BF90AF909F90CD
:102AD0008F907F906F905F904F900895009769F06E
:102AE000FC0101900020E9F73197AF01481B590B19
:102AF000BC0187E792E00C94931D80E090E008957C
:102B0000E7E7F2E022A5238F23A5248F24A5258FB4
:102B1000908F878B728F618F578F468F81E090E007
:102B200091A380A38BE792E00C94D720AF92BF9241
:102B3000CF92DF92EF92FF920F93CF93DF93EC014E
:102B40007B016A01590100FF16C0AB014F5F5F4F67
:102B5000B9016E197F09C6018C0F9D1F0E94801557
:102B6000AE014F5F5F4FB5016C1B7D0BC6018E0D33
:102B70009F1D0E94801501FF16C0A7014F5F5F4F88
:102B8000B5016E197F09C6018C1B9D0B0E94801533
:102B9000AE014F5F5F4FB5016C1B7D0BC6018E19F7
:102BA0009F090E94801503FF12C0A7014F5F5F4F6E
:102BB000B501C6018C0F9D1F0E948015AE014F5FAD
:102BC0005F4FB501C6018E0D9F1D0E94801502FF4B
:102BD0001BC0A7014F5F5F4FB501C6018C1B9D0B4A
:102BE0000E948015AE014F5F5F4FB501C6018E197F
:102BF0009F09DF91CF910F91FF90EF90DF90CF90E1
:102C0000BF90AF900C948015DF91CF910F91FF9002
:102C1000EF90DF90CF90BF90AF9008954F925F926A
:102C20006F927F928F929F92AF92BF92CF92DF92DC
:102C3000EF92FF920F931F93CF93DF932C014B01E1
:102C4000142F042F9B01AC0163E070E080E090E062
:102C50000E949615AA24A394B12CC12CD12C93E0E8
:102C6000E92EF12C2AEF622E77247A94CEEFDFEF53
:102C70008FEFC81AD80A82E0A80EB11CCA0DDB1D5E
:102C8000012F9401A201B701C6010E949615CE142E
:102C9000DF045CF4D7FDECCF81E0E81AF10882E0B4
:102CA000680E711CC60DD71DE3CFDF91CF911F9128
:102CB0000F91FF90EF90DF90CF90BF90AF909F90DB
:102CC0008F907F906F905F904F9008950C946E1549
:102CD000CF93DF932091DF023091E002281739076C
:102CE00009F4A2C0EC019093E0028093DF02FC01A2
:102CF00084918093F0023196E491E093F102FE0119
:102D00003296E491E093F202FE013396E491E0936F
:102D1000F302FE013496E491E093F402FE0135964D
:102D2000E491E093F502FE013696E491E093F60219
:102D3000FE013796E491E093F702FE013896E491A4
:102D4000E093F802FE013996E491E093F902FE0166
:102D50003A96E491E093FA02FE013B96E491E09307
:102D6000FB02FE013C96E491E093FC02FE013D96DD
:102D7000E491E093FD02FE013E96E491E093FE02B1
:102D8000FE013F96E491E093FF02FE017096E4910C
:102D9000E093000361E1CE010E94CB2090930203F7
:102DA0008093010363E1CE010E94CB209093040342
:102DB000809303038091DF029091E002892BA1F1BF
:102DC0008091FD0280930B034091FE0240930C031F
:102DD00090910A03992341F1913069F49091FF0297
:102DE000891714F490930B03809100038417E4F483
:102DF00080930C0319C03091FA022091FC02082E36
:102E0000000C990B622F022E000C770B630F711DC3
:102E100037FD7A95861797071CF4320F30930B0312
:102E2000241714F420930C03DF91CF9108950F938E
:102E30001F93CF93DF93C0E0D0E0082F10E0B801DC
:102E40000C2E02C0759567950A94E2F7617077279A
:102E500080E10E94561F61E08EE00E94561F60E0F4
:102E60008EE00E94561F2196C830D10541F7DF91B0
:102E7000CF911F910F910895CF92DF92EF92FF9221
:102E80000F931F93CF93DF937C018B016A01E901BC
:102E90001C161D0624F58091A10280939202809158
:102EA000A202809393028091A30280939402F092F5
:102EB0008F02E0928E021093910200939002D092C2
:102EC0009602C092950210929802109297028BE798
:102ED00092E00E94D72021970F5F1F4FD9CFDF913B
:102EE000CF911F910F91FF90EF90DF90CF900895B9
:102EF0000F931F93CF93DF93C4E7D2E08A810E94A0
:102F00002D1F8C0189810E942D1F000F111F802B06
:102F1000E881EF7094E0E99FF0011124E80FF11DC2
:102F2000ED5CFE4F808188838073DF91CF911F918C
:102F30000F9108958F929F92AF92BF920F931F931C
:102F4000CF93DF93CDB7DEB7A1970FB6F894DEBF6E
:102F50000FBECDBF19A2423008F44AE08E010F5DCA
:102F60001F4F842E912CA12CB12CA50194010E94FD
:102F7000A62FE62FB901CA0101501109EA3014F455
:102F8000E05D01C0E95CD801EC93232B242B252BB9
:102F900061F7C8010E946E15A1960FB6F894DEBFC6
:102FA0000FBECDBFDF91CF911F910F91BF90AF901A
:102FB0009F908F900895E0917702F09178020190B0
:102FC000F081E02D682F87E792E00994CF92DF929D
:102FD000EF92FF92CF93DF9397FF19C06B017C01B3
:102FE0008DE20E94DB17EC0166277727CB016C1975
:102FF0007D098E099F094AE00E949A178C0F9D1F38
:10300000DF91CF91FF90EF90DF90CF9008954AE04D
:10301000DF91CF91FF90EF90DF90CF900C949A17B3
:103020004F925F926F927F928F929F92AF92BF92D8
:10303000CF92DF92EF92FF920F931F93CF93DF9384
:103040007C01EB015A0129014C0183E0880E911C9F
:103050003B0183E0680E711C6701C40ED51E84E03D
:10306000C81AD1088B01020F131F0450110942E046
:10307000B301C4010E940E1641E0B301C6010E94D3
:103080000E1644E0B801C4010E940E1648E0B801D3
:10309000C6010E940E16450188E0881A9108670152
:1030A00084E0C80ED11C24E030E0A401BE01C601BA
:1030B0000E943C1724E030E0A401B801C6010E9440
:1030C0003C17920128503109BE016C5F7F4FA5016A
:1030D000C701DF91CF911F910F91FF90EF90DF908B
:1030E000CF90BF90AF909F908F907F906F905F90A8
:1030F0004F900C943C17209172023091730282170A
:10310000930760F420916E0230916F022115310512
:1031100029F0F901E80FF91F8081089580E00895F2
:103120002F923F924F925F926F927F928F929F92D7
:10313000AF92BF92CF92DF92EF92FF920F931F93C5
:10314000CF93DF9300D0CDB7DEB76C015B017A017E
:103150003A8329832C01400E511E1B01200E311E83
:103160003C01640E751E601A710A21E0621A710832
:1031700089809A80860E971E801A910A31E0831A00
:10318000910822E0A801B101C2010E94161521E0B8
:10319000A801B101C3010E94161524E0A801B401E1
:1031A000C2010E94161528E0A801B401C3010E94C3
:1031B00016153701601A710A601A710A82E0681ADE
:1031C000710889819A81801B910BFC01E01BF10B36
:1031D0008F0102501109FFEF4F1A5F0A2FEF221AD9
:1031E000320A87E7882E82E0982EF40182A5838F29
:1031F00083A5848F84A5858F508E478AB28EA18E39
:10320000778E668E11A210A28BE792E00E94D720E3
:10321000F40182A5838F83A5848F84A5858F508E2A
:10322000478A89819A810197A80EB91EB28EA18E14
:10323000778E668E11A210A28BE792E00E94D720B3
:10324000A801B101C6010E948015C7010197A8011C
:10325000B1018C0D9D1D0F900F90DF91CF911F91AB
:103260000F91FF90EF90DF90CF90BF90AF909F9025
:103270008F907F906F905F904F903F902F900C9425
:103280008015CF93DF93EC01A881B981EB01E88130
:10329000F981A217B30784F44E175F076CF4A417E3
:1032A000B5071CF4DC014D935C932E173F073CF4EB
:1032B000EB013983288303C080E090E002C081E005
:1032C00090E0DF91CF9108958EBD00000DB407FE10
:1032D000FDCF8EB508952F923F924F925F926F92DD
:1032E0007F928F929F92AF92BF92CF92DF92EF9296
:1032F000FF920F931F93CF93DF9300D000D0CDB7F1
:10330000DEB79C838B83462E8B529F4F9A83898393
:10331000FC015080EB80FC80F3EDEF0EF11CF70117
:10332000A080B180CB80DC80F1EDCF0ED11CF60106
:10333000808091800B811C810C5F1F4FF1E05F1634
:1033400001F15F1690F022E0521639F133E053128A
:103350002FC0EB81FC81E659FF4F0190F081E02DF9
:10336000C8010995880E991E23C0EB81FC81E6599E
:10337000FF4F0190F081E02DC8010995A80EB91EFC
:1033800017C0EB81FC81E659FF4F0190F081E02DE1
:10339000C8010995881A990A0BC0EB81FC81E6598E
:1033A000FF4F0190F081E02DC8010995A81AB90AD4
:1033B000EB81FC81E259FF4F91828082EB81FC819D
:1033C000E059FF4FB182A082EB81FC81E858FF4FAA
:1033D0005082EB81FC81E859FF4F808191814596B5
:1033E000E0E6E41528F4EB81FC81E457FF4F07C0C9
:1033F000F0E4F41540F4EB81FC81E657FF4F2081A7
:103400003181820F931F9C012F5F3F4FF90144913F
:10341000442309F4AFC0FC014491441103C0009758
:1034200031F4A8C0F9012491820F911DECCFAB803B
:10343000BC80FCE6AF0EB11CF501128602969183AA
:103440008083EB81FC81E358FF4F6081C5010E94BE
:103450009D20F5018087EB81FC81E258FF4F608160
:10346000C5010E949D20582EF5018187EB81FC81CA
:10347000E158FF4F9080692DC5010E949D209A94CC
:1034800066246394712CA30101C0440F9A94EAF757
:10349000382E341AEB81FC81E058FF4F9080692D63
:1034A000C5010E949D209A94930102C0220F331FF0
:1034B0009A94E2F74901252C280EEB81FC81EF5705
:1034C000FF4F4080642DC5010E949D204A949301C6
:1034D00001C0220F4A94EAF7482E421AF50180856E
:1034E000181624F0042C000C550846C0F5019484ED
:1034F0008218292D482D632D828193810E946B2093
:10350000F50193838283292D482D632D8481958134
:103510000E948420F50195838483168217828B8014
:103520009C80FBE78F0E911C6B807C802CE7620EE9
:10353000711CF4016081C5010E949D20282EF301B9
:103540006081C5010E949D20382E40E0622DC80197
:103550000E94E22041E0632DC8010E94E22061E068
:10356000C5010E949D208111F0CFF501878185154D
:1035700004F3B8CF412C512CE981FA81808181304C
:1035800039F020F0823061F4F6010BC0F60101C081
:10359000F70180819181480E591E5182408207C0F7
:1035A000F70180819181841995099183808381E05D
:1035B00090E00F900F900F900F90DF91CF911F919F
:1035C0000F91FF90EF90DF90CF90BF90AF909F90C2
:1035D0008F907F906F905F904F903F902F900895C5
:1035E000EF92FF920F931F93CF93DF937C01EA0139
:1035F0008901FB013A97EC30F10508F0E6C0EC5C7C
:10360000FF4F0C94E72F0F5F1F4F8D569F4F7C018C
:10361000CFC0C20FD31FB7C0FC01EE56FF4F808151
:103620008F3F19F061E00E94861FF701ED56FF4FB2
:1036300061E080810E94861FF701EC56FF4F808178
:103640008F3F19F061E00E94861FCFB7F8948091F8
:103650004E03811127C0E8EEF6E18491ECEFF6E12C
:103660009491E82FF0E0EE0FFF1FE054F94EA59182
:10367000B491EC91E92321F461E08AE00E94561FA5
:1036800061E08AE00E94861F8CB580618CBD8CB59C
:1036900080648CBD61E08DE00E94861F61E08BE05C
:1036A0000E94861F80914E038F5F80934E03CFBF91
:1036B0008CB58C7F8CBD8DB581608DBD8CB5837FC5
:1036C0008CBD8CB58F7D8CBD80C09FB7F8948091E8
:1036D0004E03882319F0815080934E0380914E034E
:1036E000811105C08CB58F7B8CBD10924D039FBF9F
:1036F0006CC04230510508F468C0CC0FDD1FCC0F00
:10370000DD1F25972197F1F760C0FC01EE56FF4FB2
:1037100003C0FC01EC56FF4F80818F3F09F455C078
:103720006C2F05C0FC01ED56FF4F642F80810E9475
:10373000561F4BC0842F0E94641947C0209709F47C
:1037400044C0F80180810E9464192197F7CF209727
:10375000E1F1F80180810E946419F80181810E94E1
:1037600064192197F4CF209781F1F80180810E949C
:103770006419F80181810E946419F80182810E9414
:1037800064192197F0CF0C171D07F9F0F80181910A
:103790008F010E946419F7CFF80131978081811160
:1037A0000AC0F80180810E94641921970E5F1F4FA3
:1037B000209791F70AC0813011F460E001C061E008
:1037C000F70180810E94561FECCF81E090E0DF91ED
:1037D000CF911F910F91FF90EF900895FC012589E3
:1037E0003689E25AFF4F40815181241B350B37FD4A
:1037F0000AC0349681E090E040815181241735075A
:1038000024F080E0089580E090E00895FC01238991
:103810003489E45AFF4F40815181241B350B37FD19
:103820000AC0349681E090E0408151812417350729
:1038300024F080E0089580E090E00895EF92FF92F8
:103840000F931F93CF93DF9300D000D0CDB7DEB797
:103850008C01FC01178E168EE48CF58CF1E0EF16CE
:10386000F10409F446C01CF4EF2861F0E7C052E00F
:10387000E516F10409F472C083E0E816F10409F4D6
:10388000A5C0DCC00E94EE1B892B19F4E12CF12CA1
:10389000D8C0F801238934893C832B83828D938D92
:1038A000820F931F9A838983E45AFF4F408151818D
:1038B000349620813181240F351FBE016F5F7F4F09
:1038C000CE0103960E944119892B01F32B813C8183
:1038D000F80183899489A901481B590B578F468F9A
:1038E000348B238B89819A81821B930B938F828FD8
:1038F000A5C00E94061C892B49F2F801258936894A
:103900003C832B83828D938D820F931F9A838983AF
:10391000E25AFF4F40815181349620813181240F3A
:10392000351FBE016F5F7F4FCE0103960E94411984
:10393000892B09F4ABCF2B813C81F80185899689CD
:10394000A901481B590B578F468F368B258B8981D0
:103950009A81821B930B938F828F73C00E94EE1B00
:10396000892B09F493CFF8018389948901969A836E
:103970008983228D338D821B930B9C838B83E45A26
:10398000FF4F40815181349620813181240F351FB2
:10399000BE016F5F7F4FCE0103960E944119892BB4
:1039A00009F474CF89819A812B813C81AC01421B3F
:1039B000530BF801538F428F019723893489281BB9
:1039C000390B378F268F948B838B38C0C8010E94A8
:1039D000061C892B09F45ACFF8018589968901962E
:1039E0009A838983228D338D821B930B9C838B83D7
:1039F000E25AFF4F40815181349620813181240F5A
:103A0000351FBE016F5F7F4FCE0103960E944119A3
:103A1000892B09F43BCF89819A812B813C81AC01B0
:103A2000421B530BF801538F428F0197258936892A
:103A3000281B390B378F268F968B858BEE24E394CA
:103A4000F12CC7010F900F900F900F90DF91CF9145
:103A50001F910F91FF90EF900895FC0126818081C6
:103A6000280F20834485558582859385840F951F73
:103A70009587848740855185841795073CF032816E
:103A8000230F2083841B950B9587848708950F93BC
:103A90001F93CF93DF93EC018C010C5F1F4F8C8140
:103AA0008E7F8C831E861D8681E090E09DA38CA373
:103AB000FE01E859FF4F118210823F968083ED5A34
:103AC000FF4F108231961082319610828CEA91E27B
:103AD0009C878B878FEA91E29A8789871E8A1D8A45
:103AE000C8010E946320C8010E948B21C8010E9466
:103AF0007B21FE01EF52FF4F11821082329611821C
:103B0000108232961082FF97CD55DF4F8FEF819351
:103B1000EC17FD07E1F7DF91CF911F910F91089509
:103B20000C94FD330895CF92DF92EF92FF920F93A2
:103B30001F93CF93DF936C017A018B01C0E0D0E03B
:103B4000CE15DF0589F0D8016D918D01D601ED917B
:103B5000FC910190F081E02DC6010995892B11F4AB
:103B60007E0102C02196ECCFC701DF91CF911F915A
:103B70000F91FF90EF90DF90CF900895833081F008
:103B800028F4813099F08230A1F008958730A9F0AF
:103B90008830B9F08430D1F4809180008F7D03C0EB
:103BA000809180008F7780938000089584B58F770F
:103BB00002C084B58F7D84BD08958091B0008F7759
:103BC00003C08091B0008F7D8093B00008953FB70F
:103BD000F8948091540390915503A0915603B091AD
:103BE000570326B5A89B05C02F3F19F00196A11DCC
:103BF000B11D3FBFBA2FA92F982F8827820F911D83
:103C0000A11DB11DBC01CD0142E0660F771F881FC9
:103C1000991F4A95D1F708950F931F93CF93DF9380
:103C2000DC01EA011996ED91FC911A976631710554
:103C30005CF4643171055CF56C30710549F06F30EE
:103C4000710509F44FC047C06731710501F143C0E8
:103C50004C815D819A012150310988819981280F19
:103C6000391F398328831D968D919C911E970A8157
:103C70001B81821B930B01979B838A831983088383
:103C80008E819F819D838C835F834E8324C05C964D
:103C90002D913C915D972D5F3F4F237033275D96AB
:103CA0003C932E935C971D962D913C911E975596B3
:103CB0008D919C91569753964D915C915497241BEE
:103CC000350B2150310956963C932E9355975496B7
:103CD0009C938E935397AE01CD01DF91CF911F91AD
:103CE0000F9109948A01EC01AC01455F5F4F6FE0D1
:103CF00070E009958B859C85F801938382838D857F
:103D00009E859183808381E090E0DF91CF911F9128
:103D10000F91089580E090E008950E949932CF932A
:103D2000DF936B30710599F06F30710599F06A304F
:103D30007105E1F4EC016AE070E00E94B62400979E
:103D4000C9F06CE676E1CE010E945D220CC06BE00A
:103D500070E00CC080EF90E0FA019183808380E4F2
:103D600091E09383828381E090E004C0DF91CF9162
:103D70000C94B624DF91CF910895FC01808191814C
:103D80000C943731CF92DF92EF92FF920F931F93F3
:103D9000CF93DF93CDB7DEB7A2970FB6F894DEBF0F
:103DA0000FBECDBF8C01CB01BA01F8011182108288
:103DB000138212821582148230E0AE014F5F5F4F92
:103DC0006A010E94AE32F60101900020E9F73197B6
:103DD0007F01EC18FD08F80180819181009729F09E
:103DE000228133812E153F0508F5B7016F5F7F4FA4
:103DF0000E94CF31F801009759F091838083F382BC
:103E0000E28224813581232B89F4FC0110820EC0CB
:103E100080819181009711F00E943731F801118261
:103E20001082158214821382128208C0F801F58272
:103E3000E482B601808191810E94A732A2960FB6DA
:103E4000F894DEBF0FBECDBFDF91CF911F910F91D0
:103E5000FF90EF90DF90CF900895CF93DF93282FBE
:103E600030E0F901EA5FF84E8491F901EE50F94E25
:103E7000D491F901E252F94EC491CC2391F0811111
:103E80000E94BE1DEC2FF0E0EE0FFF1FEC52F94E2A
:103E9000A591B491EC91ED2381E090E021F480E0D4
:103EA00002C080E090E0DF91CF9108951F93CF93FF
:103EB000DF93282F30E0F901EA5FF84E8491F90191
:103EC000EE50F94ED491F901E252F94EC491CC234F
:103ED000C9F0162F81110E94BE1DEC2FF0E0EE0FED
:103EE000FF1FE653F94EA591B4918FB7F8941111C5
:103EF00005C09C91ED2FE095E92302C0EC91ED2BDC
:103F0000EC938FBFDF91CF911F910895CF93DF93F3
:103F100090E0FC01EE50F94E2491FC01E252F94E82
:103F20008491882361F190E0880F991FFC01E0548F
:103F3000F94EC591D491FC01E653F94EA591B49187
:103F4000611109C09FB7F8948881209582238883E6
:103F5000EC912E230BC0623061F49FB7F894388146
:103F6000822F809583238883EC912E2B2C939FBFE7
:103F700006C08FB7F894E8812E2B28838FBFDF917E
:103F8000CF9108958E3008F08E50877020910001F7
:103F900090E4299F90011124822B80937C008091D2
:103FA0007A00806480937A0080917A0086FDFCCF4D
:103FB000809178002091790090E0922B08958F9263
:103FC0009F92AF92BF92CF92DF92EF92FF926B01DE
:103FD0007C010E94E71D4B015C01C114D104E10486
:103FE000F104F1F00E94E71DDC01CB018819990969
:103FF000AA09BB09883E9340A105B10570F321E0F1
:10400000C21AD108E108F10888EE880E83E0981EF4
:10401000A11CB11CC114D104E104F10419F7DDCFD6
:10402000FF90EF90DF90CF90BF90AF909F908F90D8
:1040300008951F920F920FB60F9211242F933F9362
:104040008F939F93AF93BF938091500390915103AF
:10405000A0915203B091530330914F0323E0230FFB
:104060002D3720F40196A11DB11D05C026E8230FB0
:104070000296A11DB11D20934F038093500390938E
:104080005103A0935203B093530380915403909132
:104090005503A0915603B09157030196A11DB11D80
:1040A0008093540390935503A0935603B093570302
:1040B000BF91AF919F918F913F912F910F900FBE24
:1040C0000F901F901895FC01EA59FF4F8AE89EE176
:1040D000918380830895213069F038F0223079F49B
:1040E000861B910967FD93950895860F911D67FDC5
:1040F0009A950895841B910947FD93950895840F1F
:10410000911D47FD9A950895213069F038F02230CD
:1041100079F4841B910947FD93950895840F911DAF
:1041200047FD9A950895860F911D67FD9A9508950C
:10413000861B910967FD93950895DC011A964C91B1
:104140001A97ED91FC911197249130E0042E02C052
:10415000359527950A94E2F7862F840F883010F45E
:10416000E22F0EC031961196FC93EE939491E92FB5
:1041700098E0941B01C0EE0F9A95EAF7E22B885065
:104180001A968C9381E090E001C0880F6A95EAF757
:1041900081508E230895FC01E60FF11D849190E07B
:1041A000982F88273196E4918E0F911D0895AC01C8
:1041B0004D5E5F4FDC011596ED91FC91169765E120
:1041C00070E009945F926F927F928F929F92AF926C
:1041D000BF92CF92DF92EF92FF920F931F93CF93F4
:1041E000DF93EC01D62EA42E8C0108591F4FF80145
:1041F000E680B780F801C084CE185C2CDC1408F48B
:104200005D2CF80184809580F4842F2D4B2D6E2D2C
:10421000828193810E946B203C012F2D4B2D6E2DAE
:10422000C4010E948420AA2031F02EA12F8B2FA13F
:10423000288F28A509C0F8012385211115C029A5BB
:104240002F8B2AA5288F2BA5298F7C8A6B8A9E8B82
:104250008D8B852D90E09B8F8A8F2F2D30E03D8FA9
:104260002C8FCE010E94D720DC1420F0DC18B394F0
:10427000E12CC0CF6D2D6E0DF8016683B782DF9102
:10428000CF911F910F91FF90EF90DF90CF90BF9053
:10429000AF909F908F907F906F905F900895CF9395
:1042A000DF93CDB7DEB728970FB6F894DEBF0FBE09
:1042B000CDBFDC0111964D915D916D917C9114976C
:1042C0004D835E836F8378871A8219821C821B82DA
:1042D0001596ED91FC911697AE014F5F5F4F6CE024
:1042E00070E0099528960FB6F894DEBF0FBECDBFDB
:1042F000DF91CF910895CF93DF93EC01AC014F5F35
:104300005F4FED81FE816FE070E00995CE01DF9196
:10431000CF910C944F21CF93DF93EC01888180FFE4
:104320000BC0ED81FE8140E050E06BE070E0CE011B
:10433000099588818E7F8883ED81FE8140E050E081
:104340006AE070E0CE010995009719F0288121609C
:104350002883DF91CF91089581E090E008956C303B
:10436000710559F06731710589F4DC011796ED91FB
:10437000FC91189767E170E00994DC01A45ABF4FE3
:1043800088E0FA0101900D928A95E1F781E090E0D2
:104390000895EF92FF920F931F93CF93DF937C01C9
:1043A000EA018A01060F171FC017D10781F0FE012D
:1043B000449150E0D7015196ED91FC91529720E045
:1043C00030E060E170E0C70109952196EDCFDF9103
:1043D000CF911F910F91FF90EF900895AB01DC01F9
:1043E0005196ED91FC91529720E030E06CE070E046
:1043F00009940F931F93CF93DF938C01EB012097C8
:1044000039F068EE73E0C8010E94EE212197F7CFE2
:10441000DF91CF911F910F910895EF92FF920F932B
:104420001F93CF93C42F8C010A531F4FAC014953E4
:104430005F4F7A0161111BC0D8013C913C2329F0E8
:10444000FA0130813C233C132EC0622F70E0DC0166
:104450005196ED91FC91529720E030E040E050E021
:1044600009959C2F9095F7018081892317C0F80149
:1044700030813C2321F0DA013C913C23A1F4462F0A
:1044800050E0622F70E0DC015196ED91FC91529763
:1044900020E030E00995F70180818C2B8083D801E2
:1044A0008C91C82BCC93CF911F910F91FF90EF90DF
:1044B00008952FE041E00C940D226F927F928F922D
:1044C0009F92AF92BF92CF92DF92EF92FF920F93A3
:1044D0001F93CF93DF938C01EB016C0188ECC80E26
:1044E000D11C66246394FE016491E62EE2942FE0D1
:1044F000E222F62FFF707F2E8E2D90E0FC01319787
:10450000EF30F10508F0CCC0E05CFF4F0C94E72FD2
:104510004E018FEF881A980AD6016C9166956170EA
:10452000C8010E945922F12CA401B701C8010E94C0
:10453000C921A72CB12C772069F08E0C9F1CF601A5
:1045400060816170C8010E945922A401B501C801AF
:104550000E94C921FFEFEF1AFF0AEA0CFB1C12C0F0
:10456000D6016C916170C8010E945922AE014F5F63
:104570005F4FE72CF12CB701C8010E94C921BFEFA2
:10458000EB1AFB0ACE0DDF1DAECFF60160816695FA
:1045900061706625C8010E945922E72CF12C772012
:1045A00039F0AE014F5F5F4FB701C8010E94C921CA
:1045B000FFEFEF1AFF0AE6CFFE013196E491672D77
:1045C00070E0762F66276E0F711DC8010E94F921D9
:1045D0000CC0FE013196E491672D70E0762F6627BE
:1045E0006E0F711DC8010E94EE2122967CCFFE0144
:1045F0003196E4903196F4902396D6016C916170D7
:10460000C8010E945922F8014389548902C0559576
:1046100047957A94E2F74E21E42FEF294E2F50E090
:10462000D8011BC0FE013196E4903196F490239698
:10463000F60160816170C8010E945922D801559627
:104640004D915C91569702C0559547957A94E2F743
:104650004E21E42FEF294E2F50E05196ED91FC9121
:10466000529720E030E060E170E0C80109953BCF4F
:10467000872D86958695813059F030F0833071F41E
:104680006370F60160830AC061702DE044E003C0EE
:1046900061702EE042E0C8010E940D22219623CFD6
:1046A000DF91CF911F910F91FF90EF90DF90CF900E
:1046B000BF90AF909F908F907F906F9008954F9292
:1046C0005F926F927F928F929F92AF92BF92CF92A2
:1046D000DF92EF92FF920F931F93CF93DF9300D05F
:1046E0001F92CDB7DEB7FC016731710509F028C113
:1046F000828D938D7C0121E0E21AF1083701F7FCED
:104700003C01759467946F0189E2C80ED11C9F012A
:104710002D5C3F4F2F01ADE54A0E511CAA24A394F6
:10472000B12C88248A94982CD6010D916D01149790
:104730004C91D9014C9310E0041B110914961C9361
:104740000E9313971896FC92EE9217971296BC92BE
:10475000AE921197C801B7010E94922FD901169607
:104760007C936E93159717FF0BC011950195110956
:1047700014961C930E93139712969C928E921197F7
:10478000D90113968D919C911497B7010E94922F95
:10479000D9011A969C938E9319971C967C926E92CF
:1047A0001B9711974C93225F3F4F2415350509F055
:1047B000BBCF8F01CF010E941E1C892B09F4C0C002
:1047C000F801C68CD78C7C2CF29658012CE5A20EF1
:1047D000B11C9E2E8F2E4681749E402D1124408345
:1047E000E084F18482859385C89EB001C99E700DD6
:1047F000D89E700D1124C701F7FC01969C013595D8
:104800002795260F371F8281938197FD06C0C90126
:10481000B7010E94922F460F05C0C901B7010E943F
:10482000922F461B4083C901B7010E94922F9587A2
:10483000848790818181890F80833E96EA15FB05EC
:1048400051F6D8015C968D919C915D9781309105D0
:1048500031F464E877E1C8010E945D2219C082301A
:10486000910509F052C0D8015396ED90FC905497F1
:104870008FEE90E08E199F0954969C938E935397D8
:1048800063E677E1C8010E945D22F801F48AE38AB9
:10489000E12CF12C6801F0E4CF0ED11C58012EE47C
:1048A000A20EB11CF801828D938DE816F90634F53D
:1048B000D801D2968C918983F60180818A83D501B3
:1048C0008C918B83D8015196ED91FC9152979E016A
:1048D0002F5F3F4F41E050E063E170E0C801099570
:1048E000892D982D0E942D1DC6010E942D1DC501E8
:1048F0000E942D1DBFEFEB1AFB0AD4CF2EE042E041
:1049000061E0C8010E940D221BC0892B19F465EAE1
:1049100077E1A1CFD8015596ED90FC9056978FE3A3
:1049200091E08E199F0956969C938E9355976FE34D
:1049300077E1C8010E945D22F801F68AE58AA8CFD6
:1049400081E090E00F900F900F90DF91CF911F9139
:104950000F91FF90EF90DF90CF90BF90AF909F901E
:104960008F907F906F905F904F900895EF92FF929D
:104970000F931F93CF93DF9300D000D0CDB7DEB756
:104980006F30710509F454C08C016031710564F415
:104990006A30710591F06B30710509F0C9C068E3A8
:1049A00077E10E945D22D2C06431710509F44DC0E7
:1049B0006531710509F469C0BBC084E690E09A8353
:1049C000898382E490E09C838B83780187ECE80EF6
:1049D000F11CD7018C9183FF0DC0D8015196ED9148
:1049E000FC91529720E030E040E050E06BE070E056
:1049F000C8010995F7018081877F8083F801EA5318
:104A0000FF4F1082D8015196ED91FC9152979E0173
:104A10002F5F3F4F40E050E06AE070E0C801099529
:104A2000009709F495C0F70120812860208390C089
:104A300080EF90E0DA0111969C938E9380E491E0F0
:104A400013969C938E93129781C00E94061C892B0B
:104A500009F47CC0C8010E94EE1B892B09F476C0C2
:104A60006AE177E1C8010E945D22F80187898983A4
:104A7000808D8A83818D8B830188F289E02D9E0150
:104A80002F5F3F4F41E050E057C00E941E1C892B12
:104A900009F45CC0F801848D958D8130910541F059
:104AA0008230910559F0892BD1F465EA77E102C093
:104AB00064E877E1C8010E945D2221C0E388F488A0
:104AC0008FEE90E08E199F09948B838B63E677E1DC
:104AD000C8010E945D22F801F48AE38A10C0E588CB
:104AE000F6888FE391E08E199F09968B858B6FE393
:104AF00077E1C8010E945D22F801F68AE58AD801B3
:104B000057968C915797898358968C9158978A839A
:104B100059968C9159978B835A964D915C915B97DE
:104B20005196ED91FC9152979E012F5F3F4F04C02B
:104B3000C8010E94AF210CC063E170E0C801099573
:104B40002EE042E061E0C8010E940D2281E090E089
:104B50000F900F900F900F90DF91CF911F910F91B9
:104B6000FF90EF900895CF93DF93EC0180916E0258
:104B700090916F020097C9F0688179816115710584
:104B800091F040917002509171022C813D81421749
:104B9000530748F00E94A7328C819D819093730245
:104BA0008093720218C00E94373188819981909356
:104BB0006F0280936E028A819B8190937102809331
:104BC00070028C819D81909373028093720219828E
:104BD00018821B821A821D821C82DF91CF91089558
:104BE000CF93DF9300D000D000D0CDB7DEB778945C
:104BF00084B5826084BD84B5816084BD85B58260E2
:104C000085BD85B5816085BD80916E008160809392
:104C10006E001092810080918100826080938100FB
:104C2000809181008160809381008091800081600B
:104C3000809380008091B10084608093B100809166
:104C4000B00081608093B00080917A00846080938E
:104C50007A0080917A00826080937A0080917A0055
:104C6000816080937A0080917A00806880937A00D6
:104C70001092C10083E08093000164E670E080E060
:104C800090E00E94DF1F809146039091470340917E
:104C900044035091450320917B022E7F20937B0299
:104CA000109285021092840221E030E030939C0241
:104CB00020939B021092E0021092DF022093EE02FA
:104CC000109241031092420310924303009711F493
:104CD0008CEA91E290938302809382025093810246
:104CE0004093800280EF9AE190938D0280938C0232
:104CF0008BE792E00E9463208BE792E00E948B2179
:104D00008BE792E00E947B2181E08093EE0210927B
:104D1000A1021092A2021092A3028BE792E00E94DD
:104D20004F2120917E0230917F0240917C02509170
:104D30007D0260E070E080E090E00E943C178FEF21
:104D40008093A1028093A2028093A30280918402A7
:104D500090918502009741F09093810280938002A8
:104D600010928502109284028BE792E00E947B21D0
:104D70008BE792E00E944F21809180029091810206
:104D800090938502809384028CE09EE1909381024F
:104D9000809380028BE792E00E947B218BE792E078
:104DA0000E944F2162E084E00E94861F62E085E05D
:104DB0000E94861F62E081E10E94861F62E080E01F
:104DC0000E94861F62E08CE00E94861F61E087E0FF
:104DD0000E94861F61E086E00E94861F61E081E0FC
:104DE0000E94861F80916800846080936800809193
:104DF0006D008C6080936D00789461E08FE00E947C
:104E0000861F61E08EE00E94861F61E080E10E94C3
:104E1000861FFF24FA94F092A102F092A202F0926F
:104E2000A30205E010E027E330E040E451E06EE14A
:104E300070E080E090E00E94901825E330E04EE3BF
:104E400051E06FE170E081E090E00E949018F092F4
:104E5000A1028AEA8093A2021092A30223E330E027
:104E60004CE351E060E270E082E090E00E943C1789
:104E7000F2E3BF2EB092A102B092A202B092A302BE
:104E800029E130E04CE350E060E070E080E090E049
:104E90000E94101829E130E04CE350E060E070E03F
:104EA00081E490E00E94101829E130E04CE350E0EA
:104EB00060E070E082E890E00E94101829E130E0A4
:104EC0004CE350E060E070E083EC90E00E9410184A
:104ED00029E130E04CE350E060E070E084E091E0F4
:104EE0000E9410188AED9AE00E94681687E090E010
:104EF0009093490380934803A5E1CA2ED12CD09208
:104F00004B03C0924A031092A1021092A202109287
:104F1000A3028FE491E00E94661688E490E09093EB
:104F2000490380934803D0924B03C0924A0383E520
:104F300091E00E94661689E890E09093490380937F
:104F40004803D0924B03C0924A0387E591E00E9448
:104F500066168AEC90E09093490380934803D092C0
:104F60004B03C0924A038BE591E00E946616BBE0BA
:104F70008B2E992493949092490380924803D09267
:104F80004B03C0924A038FE591E00E946616F092AF
:104F9000A102F092A202F092A30203E010E029E144
:104FA00030E041E450E063E270E08AEF90E00E947C
:104FB00090181BE9E12EE092A102E092A202E09299
:104FC000A30205E010E0109349030093480388EC26
:104FD00090E090934B0380934A0383E691E00E9414
:104FE0006616109349030093480385EA90E0909376
:104FF0004B0380934A0386E691E00E9466168CEA92
:1050000090E0909349038093480380E790E0909369
:105010004B0380934A03B092A102B092A202B092D5
:10502000A30203E010E029E130E04FE550E06AE53B
:1050300070E08CED90E00E94901889E691E00E946B
:1050400066168EE990E00E946816E092A102E09256
:10505000A202E092A30203E210E01093490300933E
:10506000480382ED90E090934B0380934A038DE6D2
:1050700091E00E94661610934903009348038FEA5B
:1050800090E090934B0380934A038DE891E00E9457
:1050900066168AE090E0909349038093480386EE79
:1050A00090E090934B0380934A031092A1021092D8
:1050B000A202E092A30282EB91E00E94661684E2D3
:1050C00090E00E940E0C90E09093080180930701FD
:1050D00082E290E00E940E0C082F10E0109306016F
:1050E000009305018AED9AE00E946816F092A102F1
:1050F000F092A2021092A3020130110561F4909285
:10510000490380924803D0924B03C0924A038FE533
:1051100091E00E9466168091050190910601029728
:1051200081F489E890E0909349038093480385E1F6
:1051300090E090934B0380934A0387E591E00E94AF
:1051400066168091050190910601039781F48AEC1F
:1051500090E0909349038093480385E190E0909319
:105160004B0380934A038BE591E00E9466168EE222
:1051700090E00E940E0C893409F451C06AE070E09E
:1051800080E090E00E94DF1F00E010E060E0C801D6
:105190000E94901D0F5F1F4F00331105B9F700E00B
:1051A00010E0A80160E07AE688E190E00E94F81340
:1051B000A801405F5F4F63E070E080E090E00E94F4
:1051C000F813A801405D5F4F60EE74E483EA90E05D
:1051D0000E94F8130C5F1F4F0C30110511F76091FE
:1051E000010170910201809103019091040140E45A
:1051F00050E00E94F81360E080E290E00E94901D71
:1052000061E082E290E00E94901D61E084E290E023
:105210000E94901D69E48EE290E00E94901D85E05E
:105220000E942D1F892B39F481E090E09093620257
:105230008093610204C0109262021092610280E0C9
:105240000E942D1F892B49F481E08093600280E049
:105250000E942D1F892BD9F302C01092600280E2B8
:1052600090E00E940E0C80934E0280935F020E9499
:1052700056140E945F110E942B0F4091090150911A
:105280000A0160910B0170910C012AE0CE01019698
:105290000E94C21ECE0101960E94B325CE01019646
:1052A0000E94BD1E0E94940C80E390E00E94CE13E9
:1052B00060934402709345028093460290934702A4
:1052C00080E490E00E94CE1360930101709302018C
:1052D0008093030190930401E0E88E2EE6E99E2E70
:1052E000E8E9AE2EB12C6CEDE62EF12C75EA672EB6
:1052F000712C8091610290916202019731F080914E
:105300006002882309F474C10AC18AED9AE00E9400
:1053100068161FEF1093A1021092A2021092A3022E
:10532000F0924903E09248038CE890E090934B039D
:1053300080934A038FEC91E00E94661684E290E02D
:105340000E940E0C90E09093080180930701109347
:10535000A1021092A2021092A3020E94100C80E3FC
:1053600090E00E94CE136093090170930A0180932C
:105370000B0190930C0133243A945CE8C52ED12C98
:1053800000916102109162020130110509F0B7CF5E
:1053900085E00E942D1F892B31F51092A1021092F9
:1053A000A2021092A3020E94100C8091070190911A
:1053B0000801019739F482E090E09093080180930E
:1053C000070104C0109308010093070185E00E94C3
:1053D0002D1F892BD9F33092A1021092A2021092B4
:1053E000A3020E94100C84E00E942D1F892B11F44F
:1053F0000E94E30F80915F0290914E02891751F055
:105400000E94281480914E0280935F020E945614DD
:105410000E942B0F4091090150910A0160910B01EC
:1054200070910C018091590290915A02A0915B02F7
:10543000B0915C02481759076A077B07F9F02AE028
:10544000CE0101960E94C21ECE0101960E94B32594
:10545000CE0101960E94BD1E0E94940C809109010C
:1054600090910A01A0910B01B0910C018093590217
:1054700090935A02A0935B02B0935C0280E00E947A
:105480002D1F892B09F07CCF1092620210926102CD
:105490006091090170910A0180910B0190910C01BA
:1054A00040E350E00E94F8136091070184E290E02D
:1054B0000E94901D8091090190910A01A0910B0119
:1054C000B0910C018093440290934502A093460250
:1054D000B093470280E090E00E94CE1360930901F0
:1054E00070930A0180930B0190930C018AED9AE06E
:1054F0000E9468161092A1021092A2021092A302BA
:10550000F0924903E0924803D0924B03C0924A03C1
:105510008FEC91E00E9466160E94100C31CF8AED4C
:105520009AE00E9468161092A102DD24DA94D092CB
:10553000A2021092A3028AE090E090934903809324
:1055400048030CE810E010934B0300934A0388EDE6
:1055500091E00E946616109349030093480310934C
:105560004B0300934A03D092A1021092A202109220
:10557000A30280E490E00E94CE1360930101709337
:10558000020180930301909304014AE00E949A175C
:105590008092090190920A01A0920B01B0920C0135
:1055A00060E876E988E19BE40E9486132AE040E8FF
:1055B00056E968E970E0CE0101960E94C21ECE0154
:1055C00001960E94B325CE0101960E94BD1E0E9445
:1055D000940C68EB7BE080E090E00E94DF1F3324B6
:1055E0003A944AE0C42ED12C80916002811109C006
:1055F00084E00E942D1F892B09F0D7C00E94E30F81
:10560000D4C084E00E942D1F892B11F40E94E30F67
:105610004091090150910A0160910B0170910C01B8
:105620008091590290915A02A0915B02B0915C0264
:10563000481759076A077B0709F47DC02AE0CE01A5
:1056400001960E94C21ECE0101960E94B325CE0192
:1056500001960E94BD1E0E94940C809109019091B8
:105660000A01A0910B01B0910C0180935902909313
:105670005A02A0935B02B0935C028AED9AE00E940A
:105680006816109349030093480310934B0300934B
:105690004A031092A1021092A2021092A3026091FA
:1056A00001017091020180910301909104014AE08F
:1056B0000E949A176091090170910A0180910B0173
:1056C00090910C010E94FC329B01AC0160E876E9EC
:1056D00088E19BE40E94013028E23BE64EEE5CE468
:1056E0000E94373360934F027093500280935102AF
:1056F000909352020E9473306093010170930201F3
:1057000080930301909304013092A1021092A202AF
:105710001092A302109349030093480310934B0384
:1057200000934A034AE00E949A1760E876E988E10C
:105730009BE40E94861385E00E942D1F892B09F0AF
:1057400053CF60910101709102018091030190910A
:10575000040140E450E00E94F8131092600210929D
:10576000A1021092A2021092A302D0924903C09209
:10577000480310934B0300934A0388ED91E00E9485
:105780006616109349030093480310934B0300934C
:105790004A0360910101709102018091030190918F
:1057A00004014AE00E949A171FCF80E00E942D1F3B
:1057B000892B11F40E945F118CE00E942D1F892B10
:1057C00039F085E00E942D1F892B09F089C1BAC0EC
:1057D0008AED9AE00E946816809105019091060179
:1057E000019759F51092A1021092A2021092A30201
:1057F0008BE091E0909349038093480305E110E02A
:1058000010934B0300934A038FE591E00E946616C4
:105810008FEF8093A1028093A2021092A30289E8E5
:1058200090E0909349038093480310934B030093B7
:105830004A0387E591E00E946616809105019091E8
:105840000601029759F51092A1021092A20210923D
:10585000A30289E890E0909349038093480305E10F
:1058600010E010934B0300934A0387E591E00E94F8
:1058700066168FEF8093A1028093A2021092A3027A
:105880008AEC90E0909349038093480310934B0374
:1058900000934A038BE591E00E9466168091050112
:1058A00090910601039759F51092A1021092A2025D
:1058B0001092A3028AEC90E09093490380934803EE
:1058C00005E110E010934B0300934A038BE591E050
:1058D0000E9466168FEF8093A1028093A20210921D
:1058E000A3028BE091E090934903809348031093C7
:1058F0004B0300934A038FE591E00E946616809166
:10590000050190910601019690930601809305018F
:1059100020914E022F5F233018F420934E0202C0D4
:1059200010924E02049731F481E090E090930601CA
:10593000809305010E942D0C8CE00E942D1F892B65
:10594000D9F33FCF80914C0290914D02892B09F001
:1059500052C081E090E090934D0280934C028AED1A
:105960009AE00E9468161FEF1093A1021092A20203
:105970001092A30227E130E04DE550E06BE570E0C6
:105980008DED90E00E9410181093A1021093A202D6
:105990001093A30203E010E029E130E04FE550E06E
:1059A0006AE570E08CED90E00E9490188BE191E048
:1059B00090934903809348038EE690E090934B03C5
:1059C00080934A0384E292E00E9466168CEA90E09B
:1059D000909349038093480380E790E090934B03B2
:1059E00080934A0389E691E00E9466160E942D0C7E
:1059F0000E940A106CC010924D0210924C0220902E
:105A0000090130900A0140900B0150900C018091E7
:105A1000440290914502A0914602B0914702BC0118
:105A2000CD01620D731D841D951D6093400270931E
:105A3000410280934202909343020E94FC320E94F2
:105A400086132AE0B201A101CE0101960E94C21E76
:105A5000CE0101960E94B325CE0101960E94BD1E83
:105A60008AED9AE00E9468168CEA90E090934903D0
:105A70008093480380E790E090934B0380934A0320
:105A800082E38093A1028093A2028093A30289E61D
:105A900091E00E94661603E010E029E130E04FE556
:105AA00050E06AE570E08CED90E00E949018109252
:105AB000A1021092A2021092A30227E130E04DE56C
:105AC00050E06BE570E08DED90E00E94101885E0ED
:105AD0000E942D1F892BD9F380914E020E94281419
:105AE00081E10E942D1F892B09F0E1C0F8940091FB
:105AF00007011091080102301105B9F480910901E4
:105B000090910A01A0910B01B0910C01BC01CD0153
:105B1000660F771F881F991F609355027093560276
:105B2000809357029093580208C0609109017091C8
:105B30000A0180910B0190910C010E94FC320E949D
:105B4000861384E690E090934903809348038CE8A1
:105B500090E090934B0380934A038AED9AE00E9471
:105B600068168FEF8093A1021092A2021092A302F6
:105B70000130110519F481EE91E002C08BEE91E045
:105B80000E9466168AEFD82E90E5C92E81E10E9408
:105B90002D1F1092A1021092A2021092A302892B33
:105BA00009F06EC020E130E04EE051E064EB70E0BF
:105BB00089E290E00E943C1782E10E94C21F64E4E7
:105BC00070E00E94922F603171052CF470935402A2
:105BD0006093530206C08FE090E09093540280934C
:105BE0005302209053023090540221E1522E529CD5
:105BF0008001539C100D11248DEF97E00E946816D0
:105C00001092A1021092A2021092A3028FE090E0E3
:105C100082199309589EA001599E500D1124485D88
:105C20005F4F20E130E061E970E0C80189960E9491
:105C30003C1788E290E09093490380934803709268
:105C40004B0360924A0301E010E08091530290916F
:105C50005402801791070CF499CFD092A1020A3018
:105C600011051CF4C092A20202C01092A20210926E
:105C7000A30285EF91E00E9466160F5F1F4FE5CFEC
:105C80002EE130E04AEF50E068E770E08EE190E00E
:105C90000E943C170E942D0C20E130E04EE051E0C4
:105CA00061E970E089E290E00E943C17789480916D
:105CB000090190910A01A0910B01B0910C01873F5D
:105CC0009E49A442B10514F061E001C060E081E0AA
:105CD0000E94561F80915F0290914E02891751F0E9
:105CE0000E94281480914E0280935F020E945614F5
:105CF0000E942B0F80914C0290914D020197D1F59B
:105D000080915D0290915E02092E000CAA0BBB0BE4
:105D1000409148025091490260914A0270914B02B1
:105D2000481759076A077B0711F40E9400138091F6
:105D30005D0290915E02092E000CAA0BBB0B4091F4
:105D400048025091490260914A0270914B024817F3
:105D500059076A077B0709F44DC00E942D0C0E9469
:105D60000A10809148029091490290935E028093BC
:105D70005D0240C04091090150910A0160910B0100
:105D800070910C018091590290915A02A0915B028E
:105D9000B0915C02481759076A077B0711F40E940B
:105DA00000130E942D0C4091090150910A0160914D
:105DB0000B0170910C012AE0CE0101960E94C21ED7
:105DC000CE0101960E94B325CE0101960E94BD1E10
:105DD0000E94940C8091090190910A01A0910B01FD
:105DE000B0910C018093590290935A02A0935B02E8
:105DF000B0935C0280E090E0892B09F47ACA0E949B
:105E0000000071CA8EE692E00C94BD1ECF93DF9322
:105E1000C4E7D2E083E0898382E08A8360E083E0A4
:105E20000E94861F60E08A810E94861F61E089814E
:105E30000E94561F61E08A810E94561F1882C7E7A0
:105E4000D2E01B821A828FE191E099838883CE0190
:105E50000E94471D87E291E099838883CE010E94CA
:105E6000471D8FE89EE190934503809344038FE59F
:105E700093E2909347038093460389E080930D0358
:105E80008AE080930E0388E080930F03E7EEF6E14B
:105E9000E491F0E0EE0FFF1FE653F94E85919491E7
:105EA00090931B0380931A03EBEFF6E1E491E093E8
:105EB0003403E8EEF6E1E491F0E0EE0FFF1FE65365
:105EC000F94E8591949190931D0380931C03ECEF00
:105ED000F6E1E491E0933503E6EEF6E1E491F0E0DB
:105EE000EE0FFF1FE653F94E8591949190931F0397
:105EF00080931E03EAEFF6E1E491E09336038FE22C
:105F000091E0998388834091090150910A01609141
:105F10000B0170910C012AE08EE692E0DF91CF91A7
:105F20000C94C21E97FB072E16F4009407D077FD41
:105F300009D00E94ED2F07FC05D03EF49095819585
:105F40009F4F0895709561957F4F0895A1E21A2E95
:105F5000AA1BBB1BFD010DC0AA1FBB1FEE1FFF1F0D
:105F6000A217B307E407F50720F0A21BB30BE40B5D
:105F7000F50B661F771F881F991F1A9469F76095A4
:105F80007095809590959B01AC01BD01CF0108955E
:105F9000052E97FB1EF400940E94DF2F57FD07D0BB
:105FA0000E94A62F07FC03D04EF40C94DF2F5095CF
:105FB0004095309521953F4F4F4F5F4F08959095F5
:105FC0008095709561957F4F8F4F9F4F0895EE0F8D
:105FD000FF1F0590F491E02D0994AA1BBB1B51E112
:105FE00007C0AA1FBB1FA617B70710F0A61BB70B49
:105FF000881F991F5A95A9F780959095BC01CD01EE
:1060000008950E9415300C94BB330E94B43358F0AD
:106010000E94AD3340F029F45F3F29F00C94A43383
:1060200051110C94EF330C94AA330E94CC3368F3D3
:106030009923B1F3552391F3951B550BBB27AA2741
:1060400062177307840738F09F5F5F4F220F331F7B
:10605000441FAA1FA9F335D00E2E3AF0E0E832D043
:1060600091505040E695001CCAF72BD0FE2F29D046
:10607000660F771F881FBB1F261737074807AB0718
:10608000B0E809F0BB0B802DBF01FF2793585F4F8D
:106090003AF09E3F510578F00C94A4330C94EF3302
:1060A0005F3FE4F3983ED4F3869577956795B7956F
:1060B000F7959F5FC9F7880F911D9695879597F97A
:1060C0000895E1E0660F771F881FBB1F62177307F3
:1060D0008407BA0720F0621B730B840BBA0BEE1F08
:1060E00088F7E09508950E94D43388F09F5798F080
:1060F000B92F9927B751B0F0E1F0660F771F881FCD
:10610000991F1AF0BA95C9F714C0B13091F00E94E6
:10611000EE33B1E008950C94EE33672F782F882783
:10612000B85F39F0B93FCCF3869577956795B3950D
:10613000D9F73EF490958095709561957F4F8F4F7C
:106140009F4F0895CF93DF938230910510F482E042
:1061500090E0E0915A03F0915B0320E030E0C0E072
:10616000D0E0309711F14081518148175907C0F0B4
:106170004817590761F482819381209719F09B8316
:106180008A832BC090935B0380935A0326C021150A
:10619000310519F04217530718F49A01BE01DF01C7
:1061A000EF010280F381E02DDCCF2115310509F1EB
:1061B000281B390B2430310590F412968D919C9157
:1061C00013976115710521F0FB019383828304C04D
:1061D00090935B0380935A03FD01329644C0FD0106
:1061E000E20FF31F81939193225031092D933C9339
:1061F0003AC02091580330915903232B41F4209148
:1062000017013091180130935903209358032091BE
:106210001501309116012115310541F42DB73EB716
:106220004091190150911A01241B350BE09158033C
:10623000F0915903E217F307A0F42E1B3F0B281728
:10624000390778F0AC014E5F5F4F2417350748F0EF
:106250004E0F5F1F509359034093580381939193BE
:1062600002C0E0E0F0E0CF01DF91CF9108950F93FD
:106270001F93CF93DF93009709F48CC0FC013297F2
:106280001382128200915A0310915B0301151105CC
:1062900081F420813181820F931F20915803309126
:1062A00059032817390779F5F0935903E0935803F8
:1062B00071C0D80140E050E0AE17BF0750F412960D
:1062C0002D913C911397AD012115310509F1D901AB
:1062D000F3CF9D01DA013383228360817181860FC0
:1062E000971F8217930769F4EC0128813981260FE3
:1062F000371F2E5F3F4F318320838A819B81938399
:106300008283452B29F4F0935B03E0935A0342C048
:106310001396FC93EE931297ED01499159919E01CA
:10632000240F351FE217F30771F480819181840FE8
:10633000951F029611969C938E938281938113965A
:106340009C938E931297E0E0F0E0D80112968D9125
:106350009C911397009719F0F8018C01F6CF8D915D
:106360009C9198012E5F3F4F820F931F20915803FD
:10637000309159032817390769F4309729F410929E
:106380005B0310925A0302C01382128210935903C6
:1063900000935803DF91CF911F910F910895A0E0D2
:1063A000B0E0E5EDF1E30C940F34EC01009721F43B
:1063B000CB010E94A230B8C0FC01E60FF71F9C0180
:1063C00022503109E217F30708F4ACC0D9010D914E
:1063D0001C91119706171707B0F00530110508F446
:1063E0009FC0C80104978617970708F499C0025008
:1063F0001109061B170B019311936D937C93CF0129
:106400000E9437318DC05B01A01AB10A4C01800E89
:10641000911EA0915A03B0915B0340E050E0E12C43
:10642000F12C109709F44AC0A815B905D1F56D9063
:106430007C901197630182E0C80ED11CCA14DB0462
:1064400080F1A3014A195B096A0182E0C80ED11CE0
:106450001296BC9012971396AC91B5E0CB16D1046E
:1064600040F0B282A38351834083D9016D937C9322
:106470000AC00E5F1F4FC301800F911FF901918366
:106480008083EB2DFA2FE114F10431F0D70113963C
:10649000FC93EE93129744C0F0935B03E0935A038E
:1064A0003FC08D919C9111974817590708F4AC0192
:1064B0007D0112960D90BC91A02DB3CF8091580311
:1064C0009091590388159905E1F446175707C8F4C8
:1064D0008091150190911601009741F48DB79EB7F8
:1064E0004091190150911A01841B950BE817F90787
:1064F000C8F4F0935903E0935803F9017183608362
:106500000FC0CB010E94A2307C01009759F0A80176
:10651000BE010E949E32CE010E943731C70104C0E5
:10652000CE0102C080E090E0CDB7DEB7EEE00C9483
:106530002B3481E090E0F8940C944234FB01DC01B0
:1065400002C001900D9241505040D8F70895FB01D0
:10655000DC0101900D920020E1F70895253231050C
:1065600020F4223010F00C94B932FA011082CA01E2
:106570000895BB272A3051F4992342F4BDE2909547
:106580008095709561957F4F8F4F9F4F0C94C932C6
:10659000BB27FA01A62F6217710581059105330B00
:1065A00030FB66F0AA27660F771F881F991FAA1F66
:1065B000A21710F0A21B63953850A9F7A05DAA336B
:1065C00008F0A95DA19336F7B111B1931082CA0109
:1065D0000C94EA32DC01FC01672F71917723E1F71B
:1065E000329704C07C916D9370836291AE17BF07A0
:1065F000C8F30895E89409C097FB3EF49095809500
:10660000709561957F4F8F4F9F4F9923A9F0F92F78
:1066100096E9BB279395F695879577956795B795F6
:10662000F111F8CFFAF4BB0F11F460FF1BC06F5FDC
:106630007F4F8F4F9F4F16C0882311F096E911C0EE
:10664000772321F09EE8872F762F05C0662371F00F
:1066500096E8862F70E060E02AF09A95660F771F23
:10666000881FDAF7880F9695879597F908950E9405
:106670004A330C94BB330E94AD3338F00E94B433DC
:1066800020F0952311F00C94A4330C94AA33112418
:106690000C94EF330E94CC3370F3959FC1F3950FA8
:1066A00050E0551F629FF001729FBB27F00DB11D96
:1066B000639FAA27F00DB11DAA1F649F6627B00D26
:1066C000A11D661F829F2227B00DA11D621F739F0F
:1066D000B00DA11D621F839FA00D611D221F749F1D
:1066E0003327A00D611D231F849F600D211D822F64
:1066F000762F6A2F11249F5750409AF0F1F088238B
:106700004AF0EE0FFF1FBB1F661F771F881F9150B7
:106710005040A9F79E3F510580F00C94A4330C948F
:10672000EF335F3FE4F3983ED4F386957795679512
:10673000B795F795E7959F5FC1F7FE2B880F911DE1
:106740009695879597F9089597F99F6780E870E087
:1067500060E008959FEF80EC089500240A941616D7
:10676000170618060906089500240A94121613063F
:10677000140605060895092E0394000C11F48823CD
:1067800052F0BB0F40F4BF2B11F460FF04C06F5FE9
:106790007F4F8F4F9F4F089557FD9058440F551FBF
:1067A00059F05F3F71F04795880F97FB991F61F093
:1067B0009F3F79F087950895121613061406551F0A
:1067C000F2CF4695F1DF08C0161617061806991F76
:1067D000F1CF86957105610508940895E894BB276B
:1067E00066277727CB0197F90895F999FECF92BDD7
:1067F00081BDF89A992780B50895262FF999FECF83
:106800001FBA92BD81BD20BD0FB6F894FA9AF99ACD
:106810000FBE019608952F923F924F925F926F9212
:106820007F928F929F92AF92BF92CF92DF92EF9220
:10683000FF920F931F93CF93DF93CDB7DEB7CA1BA1
:10684000DB0B0FB6F894DEBF0FBECDBF09942A88CC
:10685000398848885F846E847D848C849B84AA8474
:10686000B984C884DF80EE80FD800C811B81AA8101
:10687000B981CE0FD11D0FB6F894DEBF0FBECDBFCC
:10688000ED0108951BE0C3EEDBE004C0FE010E94B1
:0E689000E72F2196C43ED107C9F7F894FFCF39
:10689E00014059730701000100006A18000300004F
:1068AE00000300000000005C038000000000006B8D
:1068BE0019931D000000006B19931D000000006B62
:1068CE0019931D00020400030001100302000003CF
:1068DE000201000600040006050020060504004122
:1068EE00545400505245004D2031004D2032004D81
:1068FE00203300533A00503A0052495400312D2DA6
:10690E002D2D332D2D2D2D2D362D2D2D2D2D2D398E
:10691E00202B32302D34302D3630646200312D2D47
:10692E002D2D2D2D2D2D2D2D2D2D2D2D35302D2D7E
:10693E002D2D2D2D2D2D2D2D2D2D2D2D2D2D313072
:10694E0030002020202056464F20566572312E35BD
:10695E002020526166696E61642D323031360049F5
:10696E00462053657475700044445320434C4B3D90
:10697E00004F4E20414952203146004F4E20414992
:10698E0052203246002D004D756C7420465F5458CF
:10699E00203D207831004D756C7420465F54582090
:1069AE003D207832002E002020203130487A002001
:1069BE0020313030487A002020353030487A00209F
:1069CE0020316B487A00202031306B487A006B0002
:00000001FF
